:020000040800F2
:10500000B81B0020D55000088D8C00086183000873
:105010000000000000000000000000000000000090
:105020000000000000000000000000006D99000872
:10503000000000000000000011920008999A00088A
:10504000E7500008E7500008E7500008E750000864
:10505000E7500008895D0008E7500008E7500008A5
:1050600000000000E7500008B15C0008E7500008AD
:10507000E75000087D88000800000000E7500008A5
:1050800000000000E75000080000000000000000E1
:10509000E750000800000000E7500008E750000853
:1050A000E7500008E7500008E750000845A5000851
:1050B000E7500008E7500008000000000000000072
:1050C0000348854600F040FD00480047C5B8000889
:1050D000B81B00200448804704480047FEE7FEE76D
:1050E000FEE7FEE7FEE7FEE7359B0008C15000083B
:1050F00030B50B46014600202022012409E00D4670
:10510000D5409D4205D31D469540491B25469540F7
:1051100040191546521E002DF1DC30BDF0B51FB40C
:105120000646002082B005464024019100901BE015
:10513000019922460F46304600F0F0FB049A059B89
:10514000801A994110D310461946224600F0D6FB2A
:10515000361A8F410197224601200021009F00F05E
:10516000CDFB38184D4100902046641E0028DFDC3E
:10517000019B00982946324607B0F0BD03460B4319
:105180009B0703D009E008C9121F08C0042AFAD2FD
:1051900003E00B780370401C491C521EF9D2704783
:1051A000D2B201E00270401C491EFBD270470022BF
:1051B000F6E710B513460A4604461946FFF7F0FF16
:1051C000204610BD30B504460020034600E05B1CBD
:1051D000934203D2E05CCD5C401BF8D030BDF8B503
:1051E00002464A40D40F42004B0052085B089A42E4
:1051F00002D20246084611464A0023D0C30D4A0097
:10520000DDB2120EAD1A202D35DA49020126490A07
:10521000F6058A19002C00D0524220214F1B11465E
:10522000B9402A411018C20D9A4221D0002C17D043
:10523000012D08DCDA05801AD20F8019D207DBB203
:1052400000F098FBF8BDDA05801A012340001B0628
:10525000C01880185A428018CA0F1043490007E04E
:105260004908C2071143DA05801A801940088018DE
:1052700000F078FBF8BD61000122511A001BF7E72E
:105280000122D2075140AAE70122D2075040A6E7E7
:10529000024670B54A40D30FDB0740002DD04A00CC
:1052A0002AD0010E140E000212020919400A520AF5
:1052B0008418E50104465443000A120A2E045043A0
:1052C000A4194219200CC543AA18120C0125AD03DC
:1052D000521C521912047F39240400D0521C10436E
:1052E00001D44000491EC2B20C06C0092018401C5F
:1052F0004008802A02D003E0002070BD4008400032
:10530000002900DA0020184370BD70B502464A40FB
:10531000D50F40004A00ED0740085208002814D07D
:10532000002A12D0C40DD30D41020120C005520243
:10533000490A520AE41A091812187D34914201D31D
:10534000641C00E04900002C01DA002070BD00233D
:10535000914201D3891A0343400849000028F7D13C
:1053600000290AD0914202D10121C90705E09142EA
:1053700001D2012101E00121C943E005C018401913
:1053800000F0F0FA70BD420005D04200120E524209
:105390008A4201DB00207047C905081870470000E9
:1053A000F0B507460846584087B0C00F0490480043
:1053B0000E46590040084908BC1A884105D23846B3
:1053C00031461E4617460B46024658004008104319
:1053D0004CD0300D039040055900400D490D05900B
:1053E000401A0290402872DA18030121000B0905C7
:1053F0000843019004980092002805D00199524278
:105400000020884100920190029840210A1A0199D7
:10541000009800F073FA05460C466B4607CB00F087
:105420008EFAC0197141039A0E0D0023D71756400A
:105430001A467A40164344D0049A002A2DD0029A84
:10544000012A039A15DC1205C01A9141012636057E
:10545000001C7141D20F059ED20700930192029663
:105460002A46234600F0CCFA07B0F0BD3846314654
:10547000FAE71605224A0F46B218C01AB7410121B1
:105480000905001C4F4100187F4111461818794149
:10549000E20F10436D19644113E0E2076D081543F4
:1054A0006408C2071443039A01261205C01A9141E9
:1054B0003605001C7141CE07400830434908C0182A
:1054C00051412A46234600F08EFACDE7FFE70498C3
:1054D00001224000C117121A00238B410498314663
:1054E000C417381AA141EEE730B40124E407634041
:1054F00030BC55E730B40124E407614030BC4FE7CD
:105500000000E0FFF0B51FB488B00B9909980024A3
:1055100048400999C00F490049080991C0070B99F3
:105520000090490049080B9109990898A64608433C
:105530001CD00B990A98084318D009980124400000
:10554000420D4800410D099824050003000B20433B
:1055500009900B980003000B20430B9050181C4936
:105560004018002201901446104605E00020014634
:105570000DB0F0BD032801DA034600E003239C468A
:10558000C11A0AAE0AE05F0008ADED5B4F00F75BA1
:105590007D430027AA187C41491C5B1E6145F2DD52
:1055A000410004AB5A522104120C0A43240C401C43
:1055B0000828DFDB01980290009970460191009065
:1055C000059B049A0799069800F01AFAD0E70000A4
:1055D0000DFCFFFFF0B50C465C4085B0E40FE4071E
:1055E00003944C000026640859009446490802467A
:1055F0000296224321D062460A431ED06200570D14
:105600004A000E032303550D012402462C492405AC
:10561000781B1B0B360B4018234326436146009032
:105620001C46501AB44103D30098401C009002E07D
:10563000921800985B41002803DA0020014605B06B
:10564000F0BD0020012109050746864611E06446A9
:105650001D46141BB54106D36546521BB341744623
:1056600007430C43A646CD07400849082843921833
:105670005B4105460D43EAD11046184313D06046FE
:10568000194650407140084306D06046101AB34195
:1056900006D20122002306E000220123DB0702E0FC
:1056A0000122D2435310009874460105381C614111
:1056B000029C039D0019694100F095F9BFE70000C5
:1056C000FD03000070B54B005B0803430BD04B009B
:1056D0005C0D002633466542B341D417AD1AA34191
:1056E00002DB0020014670BD12053018514170BD2B
:1056F000C217C10F504010B54018CA0796230021A9
:1057000000F038F910BD10B500229623114600F0C4
:1057100031F910BD0EB5C217C10F5040CA0740186D
:105720000021054B0293019200910A460B4600F0BE
:1057300067F903B000BD0000330400000EB5054951
:105740000291002100910A460B46019100F058F9A0
:1057500003B000BD33040000C20F4100400201232A
:10576000400ADB05D207090EC0187F2901DA0020A4
:105770007047962903DC9623591AC84001E09639F0
:105780008840002AF4D04042704741004002012284
:10579000400AD205090E80187F2901DA00207047DF
:1057A000962903DC9622511AC840704796398840E2
:1057B0007047000070B5CD0F4A0009030123090BA3
:1057C0001B0519430B4BED070024520D9A4201DAD9
:1057D000002070BD074B34339A4203DC9A1A00F064
:1057E0009DF802E00449511888402C43F1D0404212
:1057F00070BD0000FF030000CDFBFFFF4A0009035E
:105800000123090B1B051943094B10B5520D9A4290
:1058100001DA002010BD064B34339A4203DC9A1A99
:1058200000F07CF810BD03495118884010BD0000FD
:10583000FF030000CDFBFFFFC20FD207400040086E
:105840000BD0C10D0723DB01C91840020905400A2E
:105850001143C208400711437047002001467047BA
:1058600010B5002904DB0124E40740428C412146A5
:10587000002B04DB1C460123DB075242A3418B4271
:1058800000D1824210BD000010B5002904DB0124C4
:10589000E40740428C412146002B04DB1C460123D7
:1058A000DB075242A341994200D1904210BD000053
:1058B000CB0FDB07490010B5490802460A4307D061
:1058C0000A0D07240903E401090B121B002A01DC5D
:1058D000002010BDC900440F0C43C100E018D205E0
:1058E000801800F03FF810BD0122D207002800DB2D
:1058F000101A002900DB511A8142704710B5202A86
:1059000004DB0146203A9140002010BD9140202345
:105910009C1A0346E3401943904010BD10B5202A5D
:1059200004DB0846203AD040002110BD0B46D3408E
:10593000D0402024A21A91400843194610BD10B54A
:10594000202A06DBCB170846203A1041C1170B432B
:1059500006E00B461341D0402024A21A9140084390
:10596000194610BD002904DA401C490001D1400845
:105970004000704770B40024050C05D110240004C9
:1059800002D1002921D01124050E01D100020834D2
:10599000050F01D10001241D850F01D18000A41C39
:1059A000002801DB4000641C002908D020252E1BA4
:1059B0000D46F540A14000D00121294308430106CE
:1059C0001B1B000ADB1D02D5002070BC7047DB05E5
:1059D000181880180029F8DA401C4900F5D170BC6D
:1059E00040084000704710B5002B08DA0024401C26
:1059F000614192185B411A4301D14008400010BD3B
:105A0000F0B51FB482B005460C0003D0084604F080
:105A100053FE02E004F050FE203002460090214682
:105A20002846FFF76BFF049B059A04460F46184370
:105A30001143084314D0184610431BD0009840214E
:105A40000A1A18460599FFF769FF05460E46009A9F
:105A500005990498FFF752FF084305D0012004E0A0
:105A60002046394607B0F0BD0020C11705430E435C
:105A70002C43374300990E986305401A7905E40AD0
:105A800000220C43FD0A0A3002D500200146E9E756
:105A90000105101969410C9C0D9D00196941FFF722
:105AA000A2FFDFE7FEB500231A461B1A8A4103DB7B
:105AB0000020014603B0F0BD4A000D0301212D0B6B
:105AC0000905520D0D43D10702D100186D41521E38
:105AD0005110FF31FF310131002704463E46384660
:105AE000009701910246012100200905FFF716FFEA
:105AF000C3197141F818324684468E464A416146C0
:105B00002846611A904104D36046241A954176468E
:105B10001F46241900986D41401C00903428E1DD97
:105B2000F91930467041091BA84103D20022D24323
:105B3000134601E00022134601980105381C71410B
:105B4000FFF751FFB6E70000064C0125064E05E0C1
:105B5000E36807CC2B430C3C98471034B442F7D38E
:105B6000FFF7B2FAB0C70008D0C7000870B58C18AC
:105B70000578401C6B075B0F01D10378401C2A118C
:105B800006D10278401C03E006780E70401C491CC8
:105B90005B1EF9D12B0705D40023521E0DD40B70C8
:105BA000491CFAE70378401CCB1A921C03E01D78CD
:105BB0000D70491C5B1C521EF9D5A142D8D30020A0
:105BC00070BD000038B50446064805490068FFF777
:105BD0008FFA604300E0401E00900028FBD138BDE2
:105BE00040420F0074010020F8B504460068816847
:105BF0008907890F012902D10168C90722D181686B
:105C0000114A10261140012500290ED1816829432F
:105C100081600120FFF7D6FF01F006F807460CE08F
:105C200001F002F8C01B0A2807D9606D3043606597
:105C3000A06D2843A0650120F8BD20680068C0431E
:105C4000C007EDD10020F8BD170000801FB50B483C
:105C500000900B4801900B4802900B480390694656
:105C60000A4805F01FF90A4A08481146083905F0A4
:105C700007F800F04DFA002004B010BDBDC50008C3
:105C800099C50008F9C50008F7C500088001002083
:105C90001000002010B500231A4603E0845CE318CE
:105CA0009BB2521C8A42F9D3D84380B210BD000087
:105CB00010B5034800F074FD024800F071FD10BDFE
:105CC000581700201017002030B5446C1C252C40BC
:105CD0000125A540046C6560046863608368102B2F
:105CE000036803D099600068C26030BD9A600068A4
:105CF000C16030BD1449012048720A4602205E325C
:105D0000507203203C3A507204200E3A50720F48F1
:105D10000D4B0078087022310870203108770C494B
:105D20005A1C087858714978997123331871597140
:105D3000203318775977107551751A461E32107531
:105D40005175107651767047D8110020200100203F
:105D50004401002010B503F0DFFD202003F092FE87
:105D6000012005F009FB002003F08CFE044805F03B
:105D7000A7F9044805F056FC002005F08BFC10BD87
:105D8000E000002083800000F8B505200121000715
:105D900000F036FF0025174C002800D06560164E35
:105DA0000221304600F02CFF00281BD1012020707A
:105DB0001248808F00280ED00127BF0200223946EA
:105DC000304600F02AFF0A2004F0CAFE01223946BC
:105DD000304600F022FF0A48656000880A214843E7
:105DE00008490880012000F043FE022000F040FE38
:105DF000F8BD00006001002000040050D80D002014
:105E00002E010020400100207047000010B5084915
:105E100000224A6107494B684C1523434B604B688D
:105E2000082423434B60C009C001026010BD00007C
:105E3000A0170020002002407FB500250C46064632
:105E4000039500F0E5FDE009029003A90196009595
:105E5000684600F075FD002804D000F0ADFD00207C
:105E600004B070BD00F0A8FD0120F9E710B50023D3
:105E700002E0C45CCC545B1C9342FAD310BD00001A
:105E800010B5214A00219069C305204804D5416915
:105E9000022319434161911593699B0505D5436917
:105EA0000124234343616302194393695B0505D5CC
:105EB0004369082423434361E301194393691B05A4
:105EC00005D543690424234343616302194393695D
:105ED0009B0405D54369102423434361630219439E
:105EE00093699B0304D5446920231C4344611943EF
:105EF0009369DB0305D54369402423434361A00232
:105F00000143916110BD000000200240A017002055
:105F100070B5054600F088FE0646184C0AE0681C7D
:105F200008D0002D04D000F07FFE801BA84201D9CC
:105F3000032070BDA069C007F1D1A069800701D519
:105F40000220A061A069C00511D4A06980050ED40B
:105F5000A06940050BD4A069000508D4A06980049D
:105F600005D4A069800302D4A069C00303D5FFF75C
:105F700087FF012070BD002070BD0000002002409E
:105F8000F8B51746002605460C4600F041FD09E02D
:105F900029460220226800F01DFD002804D1241D9E
:105FA0002D1D361DBE42F3D300F006FDBE4201D2C8
:105FB0000020F8BD0120F8BD10B5084902460020B8
:105FC000054B497905E044001C5B944203D0401C1A
:105FD000C0B28842F7D310BD6413002070000020C7
:105FE00010B500F012FE10BD10B5094801F03CF8E4
:105FF00080B2FFF7A3FB074A074BFFF783FA0022A3
:10600000064BFFF7E7FAFFF7F9FB80B210BD00007F
:10601000C4150020F853E3A59B843E4000408F4008
:1060200070B5364C3448E083354821468A7F027586
:10603000C97F417533490A780276497841763049FB
:106040000520133148720A2005F0DCFA7D20C000DB
:1060500005F0F2FA2A49002213310C2005F0BCFBAE
:1060600000210C2005F0CAFB022005F01BFB264D89
:1060700000210F2005F046FA28422063F8D0206B5B
:10608000411C37D0400434D58122D20100210F2099
:1060900005F077FB0021102005F034FA410618487E
:1060A000490E0022C73005F063FA154DC735687AEE
:1060B00005281ED102221349681DFFF783F8002826
:1060C00017D10E48AE7C66710422691C4830FFF778
:1060D00055F829461331084672000D465130FFF736
:1060E0004DF86079294642000848FFF747F8032039
:1060F000207070BD04F054FB249700007000002055
:10610000391200204401002000D027247C130020F5
:1061100010B5144C1448224610321146083904F0C8
:10612000AFFD0022114BE168A068FFF753FA104A57
:10613000104B05F0D3FC00220F4BFFF7DBF90022D8
:106140000E4BFFF7DFF9FFF7B3FB20600022134689
:10615000E168A068FFF784FB01D0206810BD002033
:10616000206010BD000000208001002000AA8F40A8
:106170006C45D9CC955BC83F0000F03F40A5E54099
:1061800010B5084800F096FA0A21064800F032FAE5
:10619000044800F01DF9800503D5024800F01AF903
:1061A00080B210BD68150020F8B52F4D00220121E6
:1061B000284600F032FDFFF7E3FFFFF7A4FA2B4E6D
:1061C0003146FFF7A2F82A4C0122A060114628466A
:1061D00000F023FD2749A068002588423EDB207897
:1061E000254F002815D02570FFF7CAFFFFF78BFA5F
:1061F0003146FFF78AF8A060FFF71EFB00223B46FE
:10620000FFF772F900221D4BFFF77CF9FFF750FBF7
:106210006060A068FFF710FB00223B46FFF764F9BF
:10622000174A184BFFF76EF906460F466068FFF7EE
:1062300003FB134A144B5242FFF764F932463B46C4
:10624000FFF7AEF8FFF734FB10496060884201DDCC
:10625000616004E0FF21C905C84200D36560606841
:10626000FFF793FAC0B2F8BD0004005000401B4491
:10627000480000200000604000000C4000E0644046
:106280003333333333B33040CCCCEC3F0000C8421F
:10629000F8B5054604464035287C0026012808D07C
:1062A00001202874206881688907890F01290ED18F
:1062B00001E00220F8BD0168C90708D0606D202107
:1062C000084360650126002028743046F8BD616DE2
:1062D000FF2201329143022211436165C16889079F
:1062E000890F0091C16889088900C16020688168B0
:1062F00092071143816000F097FC07460EE000F022
:1063000093FCC01B0A2809D9606D02218843102123
:1063100008436065002028740120F8BD206880686B
:106320000028ECDB2068C168009A1143C160606DF1
:1063300080088000401C6065C5E70000F8B506468F
:106340000D464036317C01290DD0012131740168A0
:106350008A68520709D5416D20221143416500200A
:1063600030740120F8BD0220F8BD174B6A68D805CB
:1063700047109A42154C8A6A2B6812D05B035B0B5C
:106380001A438A622968490305D5A1680143A160BF
:106390000A20FFF717FC2868800312D5A06838434D
:1063A0000EE05B035B0B9A438A622968490302D5BE
:1063B000A1688143A1602868800302D5A068B84322
:1063C000A06000203074F8BD0110000000270140DB
:1063D000406D70470068006C7047000070B50400A5
:1063E00006D0606D264600254036002802D006E023
:1063F000012070BDA5653574204600F0D3F8606DAE
:10640000C00603D421688868400705D5606D102157
:10641000084360653574EBE7606DFF2201329043FD
:1064200002221043606588688207920F5B48012A48
:1064300002D10A68D2072BD1032362689B079A42D4
:1064400005D05B429A4202D05B009A4209D10A69A8
:10645000920092080A6121680A6963681A430A6116
:106460000CE00A69920092080A6181680F22920486
:106470009143816081686268114381602168CA68C4
:1064800018239A43CA602168CA68A3681A43CA607D
:10649000816801225206914381608168A28E520672
:1064A0001143816020688168C90004D48168012299
:1064B0001207114381602068C168394A1140C160E8
:1064C0002069E168022825D00020014320462030C1
:1064D0000278037B52035B001A431143226B114382
:1064E000A26992031143E269D20311432268D3687F
:1064F0001943D160616A0A46FF3AC23A05D0A26ADE
:1065000011432268D3681943D16042780121012ADE
:1065100002D00BE00420D8E70078002823D0606D7B
:10652000202210436065A06D0843A065E06B012840
:1065300020681FD00169C90703D0016949084900D3
:10654000016120684169C908C90041612068416949
:10655000A26B11434161A565606D80088000401CFD
:106560006065002070BD2068C26801231B041A43C7
:10657000C260DBE70269FF239B009A430261206847
:106580000269236CA66C1A43636C33431A4302619D
:10659000206802690A430261D3E700000027014036
:1065A0001902FEFF10B586B0044614216846FEF7B6
:1065B000FEFD0E492068884216D10D48416B4215F8
:1065C00011434163C16A01221143C162C06A694635
:1065D00010400590022000900320019000200290BE
:1065E0000520000700F050FA06B010BD002401405D
:1065F00000100240F8B504464069254640350E4675
:1066000008280BD02068C068C00709D0606D202121
:1066100008436065002028740120F8BD082700E0C9
:106620000C2700F001FB009011E0701C0FD0002E31
:1066300005D000F0F9FA0099401AB04207D9606D10
:10664000042108436065002028740320F8BD2068F9
:1066500000683842E9D0606D012149020843606555
:106660002068C16809058A0F0C21002A1BD120224D
:10667000125D002A17D10268120714D582685307E9
:106680000122002B08DB43688B434360606D1302DB
:1066900098431043606506E0606D202318436065F1
:1066A000A06D1043A065A069002801D12068016099
:1066B0000020F8BD70B504462168002089684907AC
:1066C00021D425464035297C01291CD0012129747B
:1066D000E169012904D02046FFF786FA002811D18C
:1066E000616D0A4A1140FF220132114361650021A8
:1066F000A165297422681C21116021688A6804231D
:106700001A438A6070BD022070BD0000FEF1FFFFD9
:1067100030B5014620314A790023022A04D00422F0
:10672000C2630B71012030BD026814680E25AC43B2
:10673000146002681468640864001460446C1C22CD
:10674000144001221546006CA54045604A71184668
:106750000B7130BD70B50024014620314A79022A00
:1067600003D00421C163012418E0026813680E25D8
:10677000AB431360026813685B085B001360436CF3
:106780001C221340012215469D40036C5D604A7136
:1067900000220A71816B002900D08847204670BD15
:1067A000F0B4016C0D6801680C68466C1C2304226F
:1067B0001E401746B7402F420ED067070CD50C6815
:1067C000A40602D40C6894430C60416C19408A40C2
:1067D000016C4A60016B1AE00227B74002462F4065
:1067E0002032002F17D0A70715D50C68A40605D4B2
:1067F0000C680A25AC430C6001215171446C0221E4
:106800001C40036CA140596000211171C16A00292C
:1068100018D0F0BC08470827B7402F4212D02407F1
:1068200010D50C680E25AC430C60446C01211C4053
:106830000B46A340046C6360C16351710021117168
:10684000416BE4E7F0BC704770B504003CD01F48D2
:10685000256814212818FEF74BFC800060641C4852
:1068600020640221204620300246417129681948DF
:10687000E3680140A06866691843236933431843FD
:10688000A3691843E3691843236A1843084328603F
:106890000121A0688903884210D00D488030836AA6
:1068A000656C1C210D400F26AE40B3438362656CBE
:1068B00063680D40816AAB400B4383620020E06354
:1068C00001215171107170BD012070BDF8FFFDBF35
:1068D000000002400F80FFFFF8B504468C462030D0
:1068E00001790025012909D0012606714179002787
:1068F000012905D0077102252846F8BD0220F8BD00
:1069000002214171E763206801684908490001607C
:1069100061462046FFF7D8F9206B002820680168FF
:1069200001D00E2205E00422914301602068016835
:106930000A22114301602068016831430160DBE7EE
:10694000F8B51A4E0546307C0F46012807D00120C5
:1069500030741748FFF7DCFA010002D021E0022072
:10696000F8BD0020C04338606C6814E02046FFF793
:106970004DFA0F48FFF7CCFA01460E48426808234B
:106980009A434260426843159A434260002901D00D
:106990003C6006E08034A8686A68C0018018A042A4
:1069A000E4D8002030740846F8BD0000A01700208D
:1069B00050C30000002002400548416802221143F4
:1069C000416041680122114341600020704700008E
:1069D00000200240F8B50C4C1646207C0F460128DA
:1069E00008D0012020740948FFF792FA00250028FA
:1069F00002D006E00220F8BD65613E600348FFF763
:106A000087FA2574F8BD0000A017002050C30000CD
:106A100011484168C9070BD0EFF3108172B60F4AD5
:106A2000C2600F4AC26081F310884168C9070ED165
:106A3000416889070DD5EFF3108172B6094A0261EA
:106A4000094A026181F310884068800701D501205E
:106A5000704700207047000000200240EFCDAB8956
:106A600005040302BFAE9D8C161514137047000079
:106A700010B504494A69024202D04861FFF7F6FFA7
:106A800010BD000000040140FCB500230124A2E079
:106A900027462A469F403A406FD04D68012D05D0C9
:106AA000022D03D0112D01D0122D16D18568032699
:106AB000AC465D00AE46AE406546B543AC46CE68DA
:106AC0007546AE4065462E43866046680D79BE43E6
:106AD000ED06ED0F9D4035434560C6685F00032518
:106AE000BD40AE46AE4335468E68BE402E43C660BE
:106AF0004E68022E01D0122E14D1DE08B6003618D0
:106B00000196366A5D07B446EE0E0F25B540009635
:106B10006646AE43B4460D69009EB54066462E43B8
:106B2000019D2E6206687546AE430D79AD07AD0F27
:106B3000BD40354305604D68ED004BD5294D6E6B6A
:106B400026436E639E08284DB6007519AC46AD68A5
:106B50009E07360F0F27B740BD4305273F07B842B2
:106B600001D1002715E0214FB84201D1012710E0E3
:106B70001F4FB84202D102270BE02BE01D4FB84255
:106B800001D1032705E01C4FB84201D1052700E0E1
:106B90000627B7402F436546AF60184D2E684F68F3
:106BA0009643FF0300D516432E606E684F689643E8
:106BB000BF0300D516436E60AE684F689643FF0270
:106BC00000D51643AE60EE684F689643BF0200D50D
:106BD0001643EE605B1C0A681546DA4000D057E7A2
:106BE000FCBD000000100240000001400004005005
:106BF00000080050000C0050001C00500004014030
:106C00000069084000D001207047426913460B40DC
:106C10001B0491430B4383617047002A01D08161BB
:106C2000704781627047000001488068704700002B
:106C300068010020024881680278891881607047E5
:106C40006801002010B50848002401684022114363
:106C50000160204600F00AF8002801D0012401E07C
:106C600000F04CFA204610BD0020024070B50446EA
:106C70000D4D7D202978C000FEF73AFA01460B48F9
:106C80000068FEF735FA00F035FF002809D1042C22
:106C900007D200222146401E00F058FA00206C6006
:106CA00070BD012070BD000068010020740100204B
:106CB00070477047F8B5654CE078401CE0700120E3
:106CC0006071E08B401CE0836148008802F08CFE1C
:106CD000608AFEF718FD01467F20C005FEF715FB10
:106CE0005C4D06462968FEF77AFA28600120E16AC1
:106CF000C005814201DA084603E03046FEF7C4FAD7
:106D0000E062FF21C9050025C84200D3E562A078F2
:106D100000280BD102215048FFF772FF02004F49B3
:106D20004F4817D00022FFF778FFE56302214A4859
:106D3000FFF766FF4B4E002855D0E563B08AFEF79B
:106D4000E2FC444F3968FEF7CFFD5FD2464901208F
:106D500008705DE00122D1034148FFF75EFF608AC1
:106D6000FEF7D1FC01467F20C005FEF7CEFAE16BAD
:106D7000FEF735FA3D49E0638842D7DD39480127FF
:106D8000F926403000900A213046FEF7B1F900297B
:106D900003D132493248FFF723F902212E48FFF789
:106DA0002FFF002801D0002701E0002F12D102217F
:106DB0002948FFF725FF00280CD104F057FE009961
:106DC0000120888005F0AEFB642003F0C9FE29494C
:106DD0002748C8600A2003F0C3FE3046761EF6B28C
:106DE0000028D0D1A2E7608AFEF78DFC01467F2003
:106DF000C005FEF78AFAE16BFEF7F1F91E49E06380
:106E000088429BDB1B491A48C86097E71648057003
:106E1000708F401EFEF76CFC3968FEF765FD06D8E2
:106E2000A079002803D015490120087001E013481B
:106E30000570708FFEF767FC3968FEF755FD04D2C8
:106E4000A079002801D004F0D5FDF8BD1C01002078
:106E50008C0000206401002000040050008000002D
:106E600000000050D80D00207600002000004040B7
:106E70000400FA0500ED00E00000A04083000020BF
:106E8000704770B5040010D0022025462035A87345
:106E9000204601F0FBFCA87B032805D0204600F02B
:106EA000B9F80020A873687370BD012070BD7047E9
:106EB000704710B5044600680168C943C90708D186
:106EC0008168C943C90704D1012141602046FFF709
:106ED000F1FE20680168C943890708D48168C94365
:106EE000890704D4022141602046FFF7E1FE2068B3
:106EF0000168C943490708D48168C943490704D4D4
:106F000004214160204600F0F7F820680168C94379
:106F1000090708D48168C943090704D408214160DE
:106F20002046FFF7ADFF20680168C943C90608D4B1
:106F30008168C943C90604D4102141602046FFF787
:106F4000B8FE20680168C943890608D48168C9432E
:106F5000890604D4202141602046FFF7A9FF20685C
:106F60000168C943490608D48168C943490604D465
:106F7000402141602046FFF79AFF10BDF8B504009C
:106F800005D025462035A87B002802D006E0012048
:106F9000F8BD00206873204600F04EF80220A87368
:106FA0002068C26884466368012B01D106208243B1
:106FB00016486169814202D0072040038243002BBA
:106FC00001D1D82082431248A668024018463043B7
:106FD000676A266A3E433043A66A30431043002B5B
:106FE00002D0012B04D005E02369E2691A4300E0D6
:106FF000E2681043054A914202D0A2691143084356
:107000006146C8600120A8730020F8BDFFFF0000A2
:10701000F8F119FF10B500680549884207D1054805
:10702000816B4900490881630D2000F073F810BDA1
:10703000007C00400010024010B5006808498842FA
:107040000CD10848816BC2041143816300220121E5
:107050000D2000F07BF80D2000F06CF810BD000052
:10706000007C0040001002400068C06970470000CA
:10707000F8B504460220254620351746A8731D485A
:107080000268C3041A4302602068C2689B121A4354
:10709000C260206802690126324302612268102022
:1070A0005060206881611021204601F05FFC0328B8
:1070B0001FD02168082048602068476108212046C9
:1070C00001F054FC032814D0204601F0DFFBA87B1C
:1070D00003280ED0206881683143816020680169EF
:1070E0003143016120680169042211430161AE73DB
:1070F0000020F8BD00040140704700000448416BC7
:10710000012211434163816B020411438163704783
:1071100000100240002809DBC106C90E012088408A
:1071200003490860BFF34F8FBFF36F8F70470000B4
:1071300080E100E0002805DBC106C90E012088407F
:10714000014908607047000000E100E010B503F05D
:1071500005FB10BD02494A6882434A60704700003F
:1071600000700040024801688215114301607047B9
:107170000070004002494A6802434A6070470000BC
:107180000070004005480168022211430160044874
:10719000016904221143016130BF70470070004053
:1071A00000ED00E0F0B5154A1368154D54152D6A31
:1071B0002340ED07ED0F002B04D0002D02D0166800
:1071C000A64316601668B608B600064316600D485A
:1071D000076904263743076101290DD040BF20BF4E
:1071E00020BF0169B1430161002B04D0002D02D002
:1071F000106820431060F0BD30BFF2E7007000401F
:107200000000014000ED00E0F8B5044600780027DA
:10721000534D800671D5524E403EB06BC00004D431
:10722000B06BA9050843B06301274E480168C90542
:1072300011D40168821511430160FFF7F5FC00903D
:1072400005E0FFF7F1FC0099401A642837D845485B
:107250000068C005F5D532680321090560680A4059
:107260000140914208D08103890F032904D131687C
:10727000890301D50120F8BD2A69032109040A40C8
:1072800022D0084090421FD0207880061CD5286963
:107290002A6988430121C9040A432A612A698A4369
:1072A0002A612861C0050FD5FFF7BEFC009008E0F9
:1072B000FFF7BAFC0099411A2B48814201D90320FB
:1072C000F8BD28698005F3D561688803800F03281D
:1072D00005D132680005824301400A4332602869C3
:1072E000032261681204114008432861002F04D072
:1072F000B16B012000078143B1632078C00705D03E
:10730000E868A168800880000843E860207880076A
:1073100005D5E8680C218843E1680843E8602078D7
:10732000400706D5E868032189028843216908439C
:10733000E8602078000706D5E86803210903884340
:1073400061690843E8602078000606D5E8680321F3
:1073500089048843A1690843E8600020F8BD000063
:10736000401002400070004088130000F8B50E463F
:10737000050038D05E480068C007C00FB04214D284
:107380005B4C20684008400030432060FFF74CFC15
:10739000074605E0FFF748FCC11B564881427AD8F2
:1073A0002068C007C00FB042F4D12878524C800743
:1073B00005D5E068F0218843A9680843E060287893
:1073C000C00752D06868022806D0032807D0216879
:1073D00001280AD0890504E02168890301E02168B9
:1073E0008901002903DB0120F8BD4907F9E7E168BD
:1073F000890889000143E160FFF716FC07466868C9
:1074000002280AD0032814D001281ED029E0FFF753
:107410000BFCC11B374881423DD8E0680007800F54
:107420000228F4D121E0FFF7FFFBC11B3148814264
:1074300031D8E0680007800F0328F4D115E0FFF78A
:10744000F3FBC11B2B48814225D8E0680007800F61
:107450000128F4D109E0FFF7E7FBC11B2548814271
:1074600019D8E0680007800FF5D121480168C907E5
:10747000C90FB14217D90168490849003143016079
:10748000FFF7D2FB074608E005E0FFF7CDFBC11B85
:107490001848814201D90320F8BD15480068C0078B
:1074A000C00FB042F1D12878400706D5E068072127
:1074B00009028843E9680843E0602878000707D597
:1074C000E0680721C90288432969C9000843E060D0
:1074D00000F03AF8E168094A0906090F515CC84012
:1074E0000749086007480068FFF7C0FBF8BD0000C7
:1074F000002002408813000000100240FEC6000871
:10750000740100206C010020044805490068C96826
:10751000044A4905490F515CC84070477401002076
:107520000010024017C70008044805490068C968F0
:10753000044A8904490F515CC84070477401002017
:107540000010024017C7000870B51A4AD3681A49DC
:107550000C2018408D0004280CD04E00082810D0B4
:107560000C2810D050680004410F0120C003491CB2
:10757000884070BD1068C00601D5084670BD284619
:1075800070BD304670BD98020C4C000F205C1B0291
:107590009C0FD368641CDB0301D5314603E01268FD
:1075A000D20600D4294603F09EF822460023FDF7B8
:1075B000B5FD70BD0010024000093D000EC7000877
:1075C000FEB505007ED0FE4CE7680C20E66807405B
:1075D0000120000406402878C00747D0082F05D0B6
:1075E0000C2F0AD101200004864206D120688003B6
:1075F0003CD568680028E5D038E0012069680004BF
:10760000814203D121680143216011E00523012259
:107610001B0492049942216802D111432160F1E7D1
:1076200081432160216801400091206890432060DF
:10763000686800280DD0FFF7F7FA009005E0FFF723
:10764000F3FA0099401A64287BD820688003F6D5A5
:107650000CE0FFF7E9FA009005E0FFF7E5FA009982
:10766000401A6428F0D820688003F6D42878800770
:1076700056D50923E868042F0DD00C2F01D1002E18
:1076800009D000283CD02168994301432160FFF7CD
:10769000CBFA064628E02168490701D5002891D099
:1076A00061681F22120291432A691202114361602C
:1076B0002168994301432160FFF746FFE16809060D
:1076C0000A0F00E08BE1BF49895CC840BE490860F1
:1076D000BE480068FFF7CAFA002873D120E0FFF720
:1076E000A3FA801B0228AFD820684007F7D560684E
:1076F0001F210902884329690902084360600FE0DD
:107700002068400840002060FFF78EFA064604E03B
:10771000FFF78AFA801B022896D820684007F7D422
:107720002878C00660D5002F0CD0A86900284AD060
:107730002068FF21013108432060FFF775FA0646F3
:107740002EE0C1E02068800502D5A8690028A6D0F7
:107750006068072149038843296A084360606068BC
:10776000297F0002000A090608436060286A410B6D
:107770000120C003491C8840E16809060A0F9149AD
:10778000895CC8409049086090480068FFF76EFA2D
:10779000002817D128E0FFF747FA801B0228A2D85B
:1077A00020688005F7D56068072149038843296A66
:1077B000084360606068297F0002000A09060843E8
:1077C000606011E0E2E02168FF2001308143216028
:1077D000FFF72AFA064604E0FFF726FA801B022884
:1077E00072D820688005F7D42878794E000724D510
:1077F00068690028306910D0012108433061FFF723
:1078000013FA009005E0FFF70FFA0099401A0228DA
:107810005AD830698007F6D50FE040084000306143
:10782000FFF702FA009005E0FFF7FEF90099401A11
:10783000022849D830698007F6D42878400766D5F1
:1078400000200290A06BC00006D4A06B01210907A4
:107850000843A063012002905E480168C90511D465
:107860000168821511430160FFF7DEF9009005E021
:10787000FFF7DAF90099401A642825D855480068BE
:10788000C005F5D5FF20AA680130824203D13169D5
:107890000143316111E001218902002A07D005234B
:1078A0001B029A4203D132690A433261EFE732691F
:1078B00082433261306988433061A868002810D063
:1078C000FFF7B2F9009008E05FE0FFF7ADF901467D
:1078D0000098091A4048814257D830698005F4D58C
:1078E0000DE0FFF7A1F9009006E0FFF79DF9009980
:1078F000411A3948814248D830698005F5D4029848
:10790000002804D0A06B012109078843A063686A9E
:10791000002866D00C2F3ED00126360602282068AB
:1079200005D0B0432060FFF77FF905462FE0B04354
:107930002060FFF779F9074604E0FFF775F9C01BEF
:10794000022822D820688001F7D4E96AA86AE26890
:107950000843296BFD231B049A4311430843E0604D
:10796000206830432060FFF75FF9054604E0FFF729
:107970005BF9401B022808D820688001F7D530E069
:10798000FFF752F9401B022801D90320FEBD2068F1
:107990008001F5D425E00128F8D0E0680121090430
:1079A000AA6A014091421AD10F218904EA6A014072
:1079B000914214D1032189050840296B88420DE0CA
:1079C00000100240FEC60008740100206C01002077
:1079D00040100240007000408813000001D00120D8
:1079E000FEBD0020FEBDF8B504000ED0FF27606A82
:1079F0000537002500280AD02561656126464036F6
:107A0000A562707C002807D00AE00120F8BD6068FC
:107A1000B842F3D0E561F1E73574204600F03EF856
:107A2000022171742068026840239A430260212376
:107A3000A26860689B021A4038401043E3688A02DB
:107A40001340184323690B40217D1843C907C90F10
:107A50000843A169931019400843E169382319408C
:107A60000843216A802319400843A16A9300194002
:107A7000084321680860A0690421000C0840616A7D
:107A8000102319400843216848602068C169914368
:107A9000C1616565012070740020F8BD10B586B025
:107AA000044614216846FDF782FB1049206888428D
:107AB00019D10F48416B821411434163C16A0122FD
:107AC0001143C162C06A002110400590E02000907F
:107AD0000220019003200390029104910520694641
:107AE0000007FEF7D1FF06B010BD000000300140D6
:107AF00000100240094910B5401E884201D90120FA
:107B000010BD074C60610321081F02F027FE002012
:107B1000A06107202061002010BD0000FFFFFF00D2
:107B200000E000E0F0B502462032137E012B1ED0AB
:107B3000012515760223537606687468B3687027AA
:107B4000BC430F68274377600068AC07A04205D0AC
:107B5000084CA04202D0084CA04204D180244968BD
:107B6000A34319438160557600201076F0BD0220B2
:107B7000F0BD0000000801400014014070B5050090
:107B800005D02C462034607E002802D006E001207B
:107B900070BD00202076284600F010F802206076A4
:107BA000291D286801F0F2FF0120A077A076E07679
:107BB000207760776076002070BD000000680121AA
:107BC0008907884204D10348816B012211438163F4
:107BD0007047000000100240F8B505460446203505
:107BE000287E012817D001262E760220687622688A
:107BF00090687727FF23B8431B02984390600A6878
:107C0000502A31D00EDC202A4BD006DC002A48D086
:107C1000102A3AD145E00220F8BD302A41D0402A4E
:107C200033D136E0602A27D0702A12D00120000319
:107C3000121A2AD0824228D1CB684A688968206803
:107C400001F0DDFF20688168012292031143816009
:107C50001BE0CB684A688968206801F0D0FF216882
:107C600088683843886010E0CA684968206802F074
:107C700040F85021206806E0CA684968206802F090
:107C800049F86021206801F0C5FF6E760020287653
:107C9000F8BDCA684968206802F02BF840212068C6
:107CA000F1E711462068EEE710B586B004461421CE
:107CB0006846FDF77CFA012120688907884212D1C5
:107CC0000A49CA6A02200243CA62C96A0190014095
:107CD00005914102009100210291039104906946AF
:107CE0000348FEF7D1FE06B010BD000000100240B0
:107CF00000040050F8B5064604462036307E0D4696
:107D000001280BD0012008273076002A08D0042A49
:107D100016D0082A2AD00C2A4DD137E00220F8BD0F
:107D2000206801F07FFF2068816939438161206804
:107D3000816904229143816120688169EA6812E0C7
:107D4000206801F087FF206881690122D202114377
:107D5000816120688269012189028A4382612068E9
:107D60008169EA6812021143816124E0206801F010
:107D70008AFF2068C1693943C1612068C169042252
:107D80009143C1612068C169EA6812E0206801F08E
:107D900095FF2068C1690122D2021143C1612068A8
:107DA000C269012189028A43C2612068C169EA6807
:107DB00012021143C16100203076F8BD70B5050094
:107DC00005D02C462034607E002802D006E0012039
:107DD00070BD00202076284600F00FF80220607663
:107DE000291D286801F0D2FE0120A077A076E07658
:107DF000207760776076002070BD704770B50546CB
:107E00002C4602202034002908D004290BD0082950
:107E10000ED0627F012A10D0012070BDA27E012AFF
:107E2000FAD1A0760AE0E27E012AF5D1E07605E0FB
:107E3000227F012AF0D1207700E0607701222868B4
:107E400001F0D0FE0122286892070121904205D05E
:107E5000074A904202D0074A904204D182685207F2
:107E6000520F062A02D002680A430260002070BD49
:107E7000000801400014014070B504460D4600683A
:107E8000002201F0AFFE2068016A0C4A114203D1C2
:107E9000016849084900016001202034002D06D006
:107EA000042D06D0082D06D06077002070BDA07686
:107EB000FBE7E076F9E72077F7E700001111000013
:107EC0007047704770470000F8B502680446D069F3
:107ED00011689668814B05461D402023002D6CD00B
:107EE000F7077F4DFF0FBC460D402F4379D0254645
:107EF000C7078035002F06D0CF0504D501271762AC
:107F00002A683A432A60820708D5F20706D0276814
:107F100002223A622A6804273A432A60420708D5B7
:107F2000F20706D02668042232622A68022632430B
:107F30002A6002070AD50A461A406646324305D02F
:107F40002668082232622E6816432E60020508D584
:107F50004A0106D501222668D20232622A681A43F3
:107F60002A602A68002A30D0800606D5880604D503
:107F7000616E002901D020468847286821688968F9
:107F8000490602D42821084225D0204602F0F1F803
:107F900020688168490619D5826840218A43826039
:107FA000206F002812D04F498163206FFEF7D2FB6B
:107FB00000280AD0206F816B06E0850611D58D065A
:107FC0000FD5616E77E020468847F8BD2046FFF761
:107FD00079FFF8BD05E02046FFF774FF0020286018
:107FE000F7E7256E012D56D1C50654D5CD0652D5DD
:107FF000102616622068816825464906403500290A
:108000002ADA226F116849680904090CE1D02F8B24
:108010008F42DED9698311680968890617D401681F
:1080200032019143016020688168490849008160FC
:1080300020688168402291438160E36700202066C8
:1080400020680168B1430160206FFEF761FB288B57
:10805000698B401A81B21AE0298B6A8B891A6A8B64
:1080600089B2002AB5D00029B3D00268FF25213596
:10807000AA43026020688268520852008260E36767
:1080800000202066606620680268B24302602046D5
:10809000FFF716FF9DE7C50208D5750206D501203A
:1080A000000510622046FFF70CFF92E7050605D594
:1080B0000D0603D5A16E002985D18AE7400688D533
:1080C000480686D5116820464024A1431160836785
:1080D0000021816600F043F97BE700000F080000F3
:1080E0002001000499A0000810B5040003D0A06F7F
:1080F000002802D007E0012010BD002174200155A6
:10810000204600F027F82420A0672068016849086D
:1081100049000160204602F07FF80128ECD0606A37
:10812000002802D0204601F097FE2068416809220D
:10813000D20291434160206881682A229143816084
:1081400020680168012211430160204601F0EAFE27
:1081500010BD0000F0B587B0064614216846FDF753
:1081600026F82C493068884251D12B48416B0122B6
:10817000920311434163C16A01221143C162C06A83
:1081800000251040059003204002009002200327A4
:1081900001A9A1C104200490052069460007FEF74B
:1081A00073FC1F4C1D48A560E56081C48027E56015
:1081B000A7602020256160610002A0611848083C8A
:1081C000FEF742FB002801D0FDF71EFE3467A662D1
:1081D000144C12482146143820600320606010209F
:1081E0000831A1C16561A561E56120462562FEF700
:1081F0002BFB002801D0FDF707FEF46600220121C9
:108200001B20A662FEF7A2FF1B20FEF793FF07B01C
:10821000F0BD000000380140001002403000024074
:10822000101700205817002070B5C36F202B27D1DE
:1082300000290BD0002A09D0012483682403A3421B
:1082400006D10369002B03D1CB0701D0012070BDFB
:10825000034660331C7D012C12D001241C750023C1
:108260000366084C0368A34207D05C68240204D567
:108270001C680125AD062C431C6002F0CDF870BDD2
:10828000022070BD0048004070477047FFB50446AB
:10829000806F83B017460D4620285ED1002D0AD08E
:1082A000002F08D0A168C001814207D120690028B1
:1082B00004D1E80702D0012007B0F0BD20466030AD
:1082C0000090007D012848D0009801210175002010
:1082D000802108512120A067FEF7A6FC26464036E3
:1082E0000190378277820120A1680003814202D188
:1082F0002069002805D02F46002500990020087528
:1083000011E00027F9E700228021204602F0CAF898
:10831000002815D1002F15D02168387888627F1C7D
:10832000708A401E7082708A019B00280698009017
:10833000E9D100224021204602F0B4F8002808D0FC
:108340000320B9E728882168C005C00D8862AD1CEC
:10835000E6E72020A0670020AEE70220ACE77047E8
:10836000034D044C04A002F09DF9E560FAE700001B
:108370000400FA0500ED00E0486172644661756C26
:10838000745F48616E646C65722E0D0A0000000017
:1083900030B585B014216846FCF709FF1148818B80
:1083A000002901D10221818388B2012807D0022847
:1083B00003D100F005FCFDF749FC05B030BD0122FA
:1083C000094D940221462846FEF727FC0021012092
:1083D000029103910190009469462846FEF754FBF0
:1083E000EBE700001C0100200004005010B505243C
:1083F0002407002204212046FEF70FFC002208215A
:108400002046FEF70AFC0A2002F0B1FB01220421FB
:108410002046FEF702FC0A2002F0A9FB00220421FC
:108420002046FEF7FAFB10BD10B5052424070022F4
:1084300004212046FEF7F1FB012208212046FEF729
:10844000ECFB0A2002F093FB012204212046FEF7F8
:10845000E4FB0A2002F08BFB002204212046FEF7F9
:10846000DCFB10BDF8B50024052607462546360777
:10847000002204213046FEF7D0FB0A2002F077FBF1
:10848000012204213046FEF7C8FB6006040E0821D5
:108490003046FEF7B5FB002801D0641CE4B205208D
:1084A00002F065FB6D1CEDB2082DE1D3002F03D067
:1084B000FFF79CFF2046F8BDFFF7B6FFFAE770B55F
:1084C000052605463607002204213046FEF7A5FBA7
:1084D0000024E80901D0012200E0002208213046F2
:1084E000FEF79BFB6806050E0A2002F040FB012206
:1084F00004213046FEF791FB0A2002F038FB0022EF
:1085000004213046FEF789FB0A2002F030FB641C90
:10851000E4B2082CDDD370BD10B505242407012278
:1085200008212046FEF779FB012204212046FEF7B0
:1085300074FB002208212046FEF76FFB0A2002F0A0
:1085400016FB002204212046FEF767FB10BD10B584
:1085500005242407002204212046FEF75EFB0022AA
:1085600008212046FEF759FB0A2002F000FB0122F9
:1085700004212046FEF751FB012208212046FEF788
:108580004CFB0A2002F0F3FA10BD70B505252D074B
:108590000024012208212846FEF73FFB062002F0B6
:1085A000E6FA012204212846FEF737FB062002F0F6
:1085B000DEFA07E0641CE4B2FA2C03D9FFF7C7FF28
:1085C000012070BD08212846FEF71AFB0028F1D1D2
:1085D000002204212846FEF720FB002070BD000089
:1085E000F8B501F0D1FC01F00BFD59480068C069F5
:1085F000FDF7FAFC574C5849E082898F574E002509
:10860000002931D0E26A730355499A4202DB022203
:108610000A7000E00D700A7801218902002A05D055
:10862000012A0ED0022A10D0032A1DD1A08B0128C6
:108630002ED0022818D1464808214038FFF71CFCEC
:1086400012E0FF22F5329042F0D2A08B01281DD01B
:10865000022804D008E03046FEF7DFFA04E03C4888
:1086600008214038FFF7CAFBFDF79EFD207001216D
:10867000C9023046FEF7C4FA0127FF0300282AD0BA
:1086800038480560207A002804D007E00022E2E79D
:108690000122E0E70120207201F066FF20786328C4
:1086A00006D9002208213046FEF7B7FA012205E07C
:1086B000012208213046FEF7B0FA00220520394693
:1086C0000007FEF7AAFA244C274E4034A08C274F0F
:1086D000012803D01CE025720022EAE724486946FD
:1086E000088072B680212348FDF7A6FB002804D03D
:1086F000022269461F48FDF743FC62B61EA001F046
:10870000D1FFA58403F00EFF642002F029FAFE6079
:10871000608C012808D110486584058003F002FFB1
:10872000642002F01DFAFE60208C012806D1258409
:1087300003F0F8FE642002F013FAFE600648124AC5
:108740000188914202D1C088002800D1FE60F8BDA6
:108750008C1600201C010020D80D002000040050C1
:1087600081000020640100200400FA0500ED00E013
:10877000AAAA0000384A0008BDF8C8EBC9FDBCB67B
:10878000C4A3CABD0D0A0000AA55000008B53721D0
:10879000202000F06EF80321212000F06AF840212B
:1087A000222000F066F80821232000F062F8AA21B8
:1087B000302000F05EF80A48008FC1B2322000F08D
:1087C00058F80221332000F054F85F21202000F0F7
:1087D00050F8684600F006F80A2002F0C8F908BD13
:1087E000D80D002010B501460F2000F021F8002818
:1087F00000D0012010BD10B50446FFF78DFE3220D9
:10880000FFF75DFEFFF7C1FEE0B2FFF758FEFFF78E
:10881000BCFEFFF781FE3320FFF751FEFFF7B5FEE8
:108820000020FFF71FFE0446FFF791FE204610BD13
:1088300010B50C46FFF7DFFF2070012010BD70B5AA
:108840000D460446FFF768FE3220FFF738FEFFF7BB
:108850009CFEE0B2FFF733FEFFF797FE2846FFF7D6
:108860002EFEFFF792FEFFF772FE0A2002F07FF95C
:1088700070BD10B5FFF7E3FF012010BD10B5024831
:10888000FEF717FB10BD0000C4150020FEB504461E
:10889000002772B6334A01688B1804D13248C76882
:1088A00003208004074088680190C86800904869E8
:1088B0008E69002B08D12C4940398B6ACD042B439B
:1088C0008B628B6AAB438B62014631433CD02549B6
:1088D0002368CB4205D12449CA6803239B049A43E9
:1088E000CA6025462035002810D021680A69012376
:1088F0001A430A61216848610821204600F036F8D1
:10890000032800D1A873216808204860002E10D0E9
:1089100020680169012211430161206886611021EC
:10892000204600F023F8032800D1A8732168102006
:1089300048600C482168C14206D10B48C168032237
:10894000920491433943C160206801694908490094
:10895000016121680198886021680098C86062B64A
:10896000FEBD00000084FFBF4010024070B5064607
:108970000B480D46002409490068FCF7B9FB7D212E
:10898000C90048433168401E00D103240B682A46C1
:108990009A4301D00028F6D1204670BD204E000039
:1089A000740100201CB5002116480091144A019161
:1089B0000260C16312054260816007228263012266
:1089C00002610246C16020321170FF235170C23330
:1089D00043628162117301638161042241634261D8
:1089E000C161FDF7FBFC08480090801301906946C7
:1089F0000448FDF7A3FC00210248FDF749FC1CBD1B
:108A000000240140681500200200000408B5084851
:108A1000016B012211430163006B012110400090A2
:108A200000220A20FEF792FB0A20FEF783FB08BD16
:108A300000100240F0B587B014216846FCF7B7FB80
:108A40004748C26A04210A43C262C26A0A400592C8
:108A5000C16A80263143C162C16A31400591C16A51
:108A600001242143C162C16A21400591C16A0225E6
:108A70002943C162C06A22462840059005201C2176
:108A80000007FEF7CAF8012236493748FEF7C5F855
:108A9000002236493448FEF7C0F891210520002213
:108AA00009020007FEF7B9F83148019000270520B8
:108AB0006946029700940007FDF7E6FF0C2000903E
:108AC00011200190032003900520029769460007BA
:108AD000FDF7DAFF10206A46039591C2052069462A
:108AE0000007FDF7D1FF1120019002976946039717
:108AF00000941D48FDF7C8FF1E4801906946009587
:108B000002941948FDF7C0FFE00200906946019702
:108B100002951548FDF7B8FF1748694691C16946A7
:108B200011480397FDF7B0FF91200002694691C1FB
:108B30000520694600070397FDF7A6FF69460A4826
:108B4000019700960294FDF79FFF00220121052066
:108B5000FEF7FCFA0520FEF7EDFA07B0F0BD0000C5
:108B60000010024001020000000400500830000024
:108B700000001110000021100832000010B50F4C49
:108B80000D482060FF20053060600020A060E0609C
:108B900020616061E0610121206249026062A1619F
:108BA000A0620720E0622046FEF71DFF20680168F2
:108BB00040221143016010BD00300140F415002037
:108BC00010B58AB000240494059406940794089480
:108BD0000121184809940094019402948907039490
:108BE0000160092184604160046113494461C160EE
:108BF000FEF7C4FF01200003049004A90D48FEF70E
:108C0000EBFF0C48FFF7DAF8089408A90948099423
:108C1000FEF788FF60200090084801900294082227
:108C2000694603940348FFF765F80248FFF73CF8EC
:108C30000AB010BD4C16002093040000570200003B
:108C400000B585B014216846FCF7B1FA0E480D490D
:108C50000160E1214902416000218160C160016140
:108C600081610C22C16142610162302141620121B6
:108C7000090381634900C163FFF736FA01F06EFC16
:108C800005B000BD003801408C1600207047000080
:108C9000F0B589B00A2002F0B5FC7D20C00002F0DA
:108CA000CBFCFF4C0026A670FE482065607B0C289C
:108CB00001D30B206073FC48E670FC4D00782871EE
:108CC000FB49A079097840000843E17C890008430A
:108CD000E871E06AE870010A2972401CE06260797C
:108CE000F449A8744200C81FFE38FCF747FA6079BF
:108CF000F04982004000401960311330121DFCF72A
:108D00003DFA2A20205E002803D0EB49098A081882
:108D10006085607906214843E44DE14942192231DA
:108D20000B7AD375497A117606216972E349DC4AD8
:108D30000978A972217F297329461339937F0B750E
:108D4000D27F4A75002213311C3002F045FD607954
:108D50000621484300211C3002F050FD022002F0A1
:108D6000A1FC0026EE71E673A67201252573E6725A
:108D7000D348FEF779F960840746E6706079FCF71E
:108D8000DDFCD04AD04BFCF7BDFB01F085FE002294
:108D9000AB07FCF705FBFCF731FD0006C00CC01962
:108DA00080B2E903A084884201D3401AA084C74856
:108DB000E0632079401C2071C148FEF755F9BD4F92
:108DC0002084643FC6E1BE48FEF74EF92084C04EC1
:108DD0000BE0BB48FEF748F980B22084A18C8842A2
:108DE00003D3BC4A8918884206D300210F2002F021
:108DF00089FB30422063ECD0206B411C1FD0400423
:108E00007DD58122D20100210F2002F0BAFC7D2005
:108E1000C00002F011FC002002F0C3FB0021102072
:108E200002F070FB4106A348490E26460022643832
:108E3000E16402F09DFB787A0728C3D101E001F0DC
:108E4000AFFC0222A449781DFCF7BCF90028B9D177
:108E500002F025FDF165B06502F00EFD7166306629
:108E6000F0786946401CF07092486B38027A0A70BC
:108E7000407A487008880290F18B88427ED18B48F6
:108E8000964E8C30C08E8949308085488C31098F50
:108E900041838B48FEF7E8F8208402F045FAFF2270
:108EA000216E5204606E0023891858410206080A98
:108EB0001043410849000090080E0902A166E066CF
:108EC0007A48E36D0A30A26D02F0BEFC6079636EF1
:108ED00081007648226E0818163002F0B5FC7348FF
:108EE000E36E1230A26E02F0AFFC704808214172AE
:108EF000A07C002815D002227749781D00E01CE1F3
:108F0000FCF760F900280CD16848E573C571E06C86
:108F100068491638C2B24E3908462274EA30FCF766
:108F20002DF960790022800060491C3002F054FC69
:108F30006079002180001C3002F060FC009802F093
:108F40005AFB012002F0AEFB207202216448FDF7BB
:108F500057FE00287ED000215548564B01705349DA
:108F60004F488C314A8E0287898E4187A06B6033CF
:108F7000E0631860FB7C1807000F00E07BE003282B
:108F800000D060741809A07400202071444BA572B1
:108F90009A87D987E572618B524AFF31C33189B212
:108FA000618391420BD952428918618331887D22B5
:108FB000491C89B2D2003180914200D3308036887A
:108FC0007D20C000618B70434018206407904648A4
:108FD000302107784548A77300884843FCF793FB86
:108FE00000900A2031464143A08B30220690504326
:108FF000081AFCF77DFB0099FCF787F97F21C9056A
:10900000FCF7EDF8FCF7C1FB80B237497F1E088002
:10901000B84200D1E572E6841620205EFCF77AFBA8
:1090200006460F46208CFCF789FB314A314BFCF792
:1090300069FA054603910798FCF76CFB2A46039BE7
:10904000FCF752FA3B463246FCF7AAF9FCF7B2FBB2
:10905000606400E006E0069800F0C6FC207A002874
:1090600002D080E0012177E700210F2002F04AFAC8
:109070000006F9D577E0FCF79FFF0E4A03219032F6
:109080001154FF3A06491D3A538E0B87928E4A8738
:10909000084980003031054A41188C3201902BE09C
:1090A000700000203F420F001C0100204C120020E5
:1090B0006001002064130020180E00202E01002003
:1090C000C4150020B81E85EB51B8CE3FA086010024
:1090D00000D02724983A0000440100205C010020C1
:1090E00000040050E70300003A0100203E01002088
:1090F000F853E3A59B843E40928F0A803E49B26BB1
:1091000041184A603D49736E40181630326E02F0C5
:109110009BFB316DB06B884200DA3065364A0199AD
:10912000303A5158814215DD002913D0002811DD55
:109130000298F083022030700CE0324600210F20AC
:1091400002F01FFB6079E178401C814202D00020D0
:1091500002F027FA208CA18C884200D233E6284AFC
:1091600089188842FAD8A07A012801D00220A0727A
:1091700002F0DAF8234A00210F2002F002FBE07B24
:1091800000281ED01C493C310B7848788A78022B85
:1091900017D110280CD0C82813D21B4BC91C181883
:1091A000FBF7ECFF03F0BEF9642001F0D9FC46E6C2
:1091B000164D28684000000E03D1C878FCF7A3FACA
:1091C00028600D4D0020603D2E46227863791836C8
:1091D00007E041006F5A715A8F4200D00222401CB2
:1091E000C0B29842F5D32270064A002180320F2087
:1091F00002F0C7FA09B0F0BDC41300204C120020E1
:10920000983A000000D02724D80D00204801002003
:1092100070470000F0B58DB0002005900A2002F0E4
:10922000F1F97D20C00002F007FABF4800218170EB
:10923000C26ABE4C521CC2620175214613310991AB
:10924000BB4907912146223026465A3103903136D8
:1092500020461338B74F02910690B34D0F21B64800
:10926000697100782071B54AA879127840001043DE
:10927000EA7C92001043E071A88DE070000A207231
:10928000A17429461E227C310998FBF777FF402202
:109290003046AB49FBF772FF0798698D008A40188A
:1092A0006885039902980A7AC274497A017509207F
:1092B0006072A4480078A072287F2073287D410046
:1092C00028467C30091806980A7802754978417555
:1092D00076200022954902F07FFA687906214843FA
:1092E00000211C3002F08AFA022002F0DBF9002192
:1092F0000F2002F007F938422863F8D0286B411C90
:1093000018D040047ED58122D20100210F2002F026
:1093100038FA0021102002F0F5F841068348490E82
:109320000022B43002F024F98048B430417A022996
:1093300002D0D1E001F034FA02228349401DFBF74C
:1093400041FF0028F5D178480222007D410076488F
:109350007C3009187548B530FBF734FF0028E8D198
:1093600002F09DFA704DE965A86502F085FA69661C
:1093700028660598002844D1012005906B48734D5C
:109380008C30C08E6949288067488C31098F4183B1
:109390006F48FDF769FE64496E4A0884488BFF30C8
:1093A000C33080B2488390420CD95242801848831F
:1093B0002888684A401C80B20B322880904201D332
:1093C0000020288028887D22D2004B8B4243D2186F
:1093D0000A64614A1288D3B2944602460A3A12B22B
:1093E0008B730A85002A03DA7D25ED0052190A8560
:1093F0005B1E9C4501D10122CA72C884888B00F093
:10940000F3FA00E089E0494869468C30428E0A80D0
:10941000808E488045490422B531C81FFF38FBF7CC
:10942000ADFE4148464A007D0099800011503E48FB
:10943000FF23016E406E5B040022C91850410006F4
:109440000D0A0543284602F0D6F868084000020ECF
:10945000010235480025C2668166C36D826D3348BE
:10946000483802F0F1F93048436E026E2F48443814
:1094700002F0EAF92C48C36E826E2C48403802F0A4
:10948000E3F92A49002252393C2002F0A5F90021D3
:109490003C2002F0B3F9012002F004F922490872DD
:1094A00008468078401C887001210520C903000708
:1094B000FCF796FD1C48007A002805D100210F20FA
:1094C00002F020F80006F9D5802200210F2002F0DA
:1094D00058F915494D7002E01349012048701248AF
:1094E000017D491CC9B201750F2900D2B5E6059866
:1094F000002810D10C481949828B002A02D00B8811
:109500009A4201D9098881831549808B0988401EB8
:109510004843144908800DB0F0BD134A00210F20C4
:1095200002F02FF9D8E70000700000204C12002054
:10953000180E002000D027241C010020600100200C
:10954000501400202E010020440100205C01002066
:10955000C4150020E70300003A0100202A01002082
:10956000280100202601002000902724F8B5334967
:109570003148086002F07AFA314800F0F5F9314CD0
:1095800020832F48801C00F0EFF960832C48001DD9
:1095900000F0EAF9A08387212B4889004180014629
:1095A00040310A79294F1206120EA27006D1C780E7
:1095B0000122C2870A2242870022828702890A8208
:1095C000234AC18E1170C18FA171818FE171817A9F
:1095D000217185880521A562A181C6883046FBF7E7
:1095E00087FDE08101462846FBF782FD88000818C8
:1095F00085B2164865816843FCF7A0F8154A164BFA
:10960000FBF7E8FFFCF7FAF82082A58231463846DE
:10961000FBF76EFD60820146C820FBF769FD6084A0
:109620000120E083FCF7E0FCE082228A0B490C4831
:10963000FDF71EFDF8BD000095A50008680000209C
:10964000004F00081C010020D80D0020E803000096
:1096500018000020F853E3A59B843E40FF7F0000E4
:10966000C4150020F0B59A4D85B001202880994F8F
:10967000C820994C3880E079401CE071C00706D0C2
:10968000A08B411EA183022801D2C820A083A08BF9
:1096900000F0AAF90A2001F0B5FF7D20C00001F01A
:1096A000CBFF02218D48FDF7ABFA00283FD0002008
:1096B0008B49800009788C4E490008438949097814
:1096C0000843B072102070728848C1887D20C000A5
:1096D000FBF70EFD7073864884490078B0733046FE
:1096E0000B308A780270C97841708049421C203161
:1096F0000B7ED370497E11717C49D01C22310B7EC8
:109700005371497E9171794940310A7C0271497CDB
:10971000417100223146172002F05EF80021172027
:1097200002F06CF8022001F0BDFF724E03E0012050
:10973000BEE7FEF755FF00210F2001F0E3FE3042A7
:109740002063F6D0206B411C7ED040047DD5812261
:10975000D20100210F2002F014F80021102001F0A6
:10976000D1FE41066048490E0022B430E16401F0A8
:10977000FFFE5D4EB436707A112866D102225E4932
:10978000701DFBF71FFD00285FD1F01F027A6946AC
:109790000A70407A4870B17A2980C820FBF7A8FC8B
:1097A0003880307BA0833046544D2838C08E2880C6
:1097B000314649482839098F41835148FDF754FC07
:1097C00080B220840390608B4E49FF30C33080B25A
:1097D000608388420CD949424018608328884949EF
:1097E000401C80B20B312880884201D300202880A1
:1097F0002D887D20C000618B684340182064029052
:109800004148067828460A3800B2A6732085002809
:1098100003DA7D21C900401820853888302148436B
:10982000FBF771FF07462820205EFBF761FF3946F2
:10983000FBF76BFD7F21C905FBF7D1FCFBF7A5FF0B
:10984000314980B2088001E03FE03CE0761EB04242
:1098500001D10120E072E5841620205EFBF75AFF5B
:10986000074601910398FBF769FF284A284BFBF74D
:1098700049FE05460E460298FBF74CFF2A46334642
:10988000FBF732FE3A46019BFBF78AFDFBF792FF9E
:10989000606468460088E08313481349B430807CD4
:1098A000C7316071420008460D465130FBF766FC37
:1098B0006079294642001748FBF760FCA08BFF281F
:1098C00001D00320207005B0F0BD00F069FF00005A
:1098D0002E0100203E0100207000002000040050F6
:1098E00022010020230100204C120020D80D00206E
:1098F0001800002000D02724440100205C01002033
:10990000C4150020E70300003A010020F853E3A546
:109910009B843E407C13002070B586B014216846BD
:10992000FBF745FC01250F4EED030022294630468A
:10993000FDF773F901200024019002946946009517
:1099400003943046FDF7A0F8032001900294694685
:10995000009503943046FDF797F8022001F000F9D6
:1099600006B070BD000400500088704770470000CA
:10997000F8B5044600206A461080194D55222A7019
:10998000AA226A700322AA70661DEE702A7169719C
:10999000144A49008918AC712246E81DFBF7EEFB1A
:1099A000002007E029186A468978128889186A46D3
:1099B0001180401CB042F5DB611DA81CFCF76AF960
:1099C00001466846018029190078C87168464078C8
:1099D000087221460931024800F0ECFBF8BD000096
:1099E00004150020D80D002010B51F481D4C807DA7
:1099F0001E4960700880618A01E0521AE283E28B9E
:109A00008A42FAD2618C93B24B431B182384132AE7
:109A100002D1514308182084208C3021484364210E
:109A2000643048431249A0630968401A4B21090178
:109A300040186063FBF76EFE0E4A0F4BFBF7CAFD42
:109A4000FBF7B8FE0D492063884202DD4A428018C8
:109A50002063002801DA4018206309490968486139
:109A600010BD00001C010020D80D00208C0000203B
:109A7000B4000020F853E3A59B843E40FF7F000024
:109A8000C4150020034A1168382389B29943014361
:109A9000116070470030014010B5FDF7CBF810BDE4
:109AA00010B59AB034216846FBF781FB14210DA84C
:109AB000FBF77DFB1C2112A8FBF779FB1B48016813
:109AC0000324E402A143C21489180160FDF74AFB94
:109AD00017480169A143016106200090FF20013071
:109AE000029001200390102004900220099040046D
:109AF0000B90000100240C900A946846FDF760FD6D
:109B00000F200D9003200E900F94109401211194BA
:109B10000DA8FDF72BFC81201290032080041890E3
:109B2000149412A8FDF770FB1AB010BD007000402D
:109B30004010024010480168821511430160C1685D
:109B40000E4A1140C16001680D4A114001608168F0
:109B50004908490081600168012292049143016033
:109B6000C168FD2212049143C160002101610649D0
:109B70000448886070470000001002400C40FF88D5
:109B8000F6FFF6FE0050000800ED00E070B5026838
:109B900001239B07114C124D984203D0A04201D0E3
:109BA000A84203D17026B2434E683243984203D094
:109BB000A04201D0A84204D103231B029A43CB68E0
:109BC0001A4380239A430B691A4302608A68C2626F
:109BD000096881620121416170BD000000080140F7
:109BE0000014014010B5CB06DB0E0121046A994038
:109BF0008C430462016A9A401143016210BD30B582
:109C00008468FF252D021B021343AC430B432343FF
:109C1000836030BD826870239A430A4307210A4358
:109C20008260704730B5026A520852000262026ACE
:109C3000456883697024A3439C080B68A4002343F0
:109C40000224A2438C6845601443836149684163E0
:109C5000046230BD30B5026A10239A430262036A7F
:109C60004568826973242402A2430C6824021443C9
:109C7000202293438A68456012011A43846149682F
:109C80008163026230BD30B5026AFF2301339A431B
:109C90000262026A4568C3697024A3439C080B688A
:109CA000A400234301246402A2438C68456024027B
:109CB0001443C3614968C163046230BD30B5026AB0
:109CC00001231B039A430262036A4568C269732435
:109CD0002402A2430C68240214430122520393433A
:109CE0008A68456012031A43C461496801640262CC
:109CF00030BD30B5036A046A640864000462846994
:109D0000F025AC43120122430A24A3430B43826192
:109D1000036230BD30B5036A1024A3430362846933
:109D2000036A0F252D031203AC432243A024A3434F
:109D3000090119438261016230BD0000F8B51026A7
:109D400005252D07AE62AF20800000F010FFFCF764
:109D5000DFF9364834490068FBF79AFAFBF7FCFC58
:109D6000334C6085AE6101F0E1FB324F324E6065ED
:109D70000EE001F0DBFB6065FEF732FC606B411C1E
:109D80006163142804D92DA000F08CFC2F48C76013
:109D9000606DB042EDD10026666320780127FF0395
:109DA000030000F0B8FC05040C192D30320001222C
:109DB00039462846FCF731FFFFF754FC06E0012244
:109DC00039462846FCF729FFFFF724FA00223946D6
:109DD0002846FCF722FF18E0607A0122401E6072DC
:109DE00039462846FCF719FFFCF71AF900223946D4
:109DF0002846FCF712FF607A002806D1267004E09E
:109E0000FEF746FF01E0FFF705FA02211048FCF7D4
:109E1000F7FE002805D000200E49087001F06CFA0A
:109E2000F8BD0120F8E700000000C8420000002053
:109E3000700000200400FA053001CADE44572049B2
:109E400044204552524F522E0D0A000000ED00E012
:109E5000000400506001002010B5818CC90707D0B4
:109E600001684A6801235B049A43836A1A434A6083
:109E7000818C890707D501684A6801231B049A432E
:109E8000C36A1A434A60818C490707D501684A684A
:109E900001239B049A43036B1A434A60818C090790
:109EA00007D501684A680123DB039A43436B1A43D1
:109EB0004A60818CC90607D50268916801231B039B
:109EC0009943836B19439160818C890607D501689A
:109ED0008A6801235B039A43C36B1A438A60818CAF
:109EE000490612D503685A6801210905046C8A43A2
:109EF00022435A60026C8A4207D1026851680323E8
:109F00005B059943436C19435160818C090607D561
:109F100001684A680123DB04806C9A4302434A606B
:109F200010BD0000F8B50446002680300660FCF73E
:109F30007BFE054620680068124F000709D5012105
:109F40002B46002249052046009700F0ABFA002876
:109F50000DD12068006840070BD501212B46002257
:109F600089052046009700F09DFA002801D00320C3
:109F7000F8BD2020A067E0672666603426750020C3
:109F8000F8BD0000FFFFFF01F8B5184CC826E078C7
:109F9000002829D16079002826D101206071144D54
:109FA000686B002700281ED0686BC821081A15E0CE
:109FB0001048E168405C616988470F480A210088C1
:109FC00048430E490880E068401CE060E068C8280B
:109FD00000DBE760696BC820401A761EE1688142A9
:109FE00001D0002EE4DC6771F8BD000054000020B1
:109FF00000000240100D00202E0100204001002032
:10A0000070B5224CE07800283FD1207900283CD15F
:10A01000012020711E4EF16900250906002933DA5E
:10A020002156625791420AD1F06940062CD5A07999
:10A03000002829D0A5712089401C208124E0A17925
:10A04000002903D1A0710A2000F091FD00202056C4
:10A05000CC2148430F494218206912181279B26284
:10A06000401C00222061A256CC235A4389588142C9
:10A070000ADC25612078401C207020780E2800D151
:10A080002570A078401CA070257170BD5400002080
:10A0900000380140E801002010B5806A0022014626
:10A0A00040314A834A82FDF70DFF10BD70B5846AC6
:10A0B000A06FE56F2168896800260906002906DA85
:10A0C000212804D152200653204600F06BF8206866
:10A0D0008068400606D5222D04D15A20065320461A
:10A0E00000F047F8204680300168102211430160DB
:10A0F0002046FDF7E7FE70BD10B501460968806A8D
:10A10000096889061CD400225A210A5201680A688B
:10A11000FF2301339A430A6001688A68520852009B
:10A120008A6001688A6840239A438A602021C16757
:10A13000016E012904D101680A6810239A430A605C
:10A14000016E012902D0FEF79FF810BD5821095A6F
:10A15000FDF7B6FE10BD10B5806A016E012902D070
:10A16000FEF793F810BD5821095A4908FDF7A8FEDB
:10A1700010BD01680A68FF2321339A430A60016811
:10A180008A68520852008A60016E012904D1016870
:10A190000A6810239A430A602021C16700210166E2
:10A1A0004166704701680A68C0239A430A6020210B
:10A1B0008167704770B5164CE278002A0CD122797D
:10A1C000002A09D10122E2700025C82903DC0222FD
:10A1D000A256002A01DCE57070BD0123E356CC22B3
:10A1E00053430C4AD1500123E356CC2673439B18AA
:10A1F0000A460146181DFAF7C1FF6078401C6070DE
:10A2000060780E2800D16570A078401EA070E2E74B
:10A2100054000020E8010020F8B504460168806879
:10A220002369E66918436369002533431843724A7A
:10A230000B68724E334003430B6021684868032368
:10A240001B039843E368184348602168A069914262
:10A2500001D0236A18438B680B263602B3430343AD
:10A260008B606749236867488B420CD1C0688007C0
:10A27000800F06D0012839D0022835D0032821D1FB
:10A280001EE001271FE060498B420AD1C0680C2103
:10A29000084027D0042829D0082825D00C2811D11F
:10A2A0000EE093420ED1C16803208002014019D014
:10A2B00001208002091A19D0091A15D0814201D152
:10A2C000082700E010274F49504840398600934244
:10A2D00032D1002F0CD0022F0DD0042F10D0082F18
:10A2E0007FD126E00027EEE70227ECE70427EAE724
:10A2F000FDF70AF906E00968C90605D4304603E00F
:10A30000FDF722F9002872D062685100511881428D
:10A3100067D81103814264D3010E0602500800235E
:10A3200030185941FAF7FAFE03210902411A384A56
:10A3300055E00120C003E7E70122E369D20393421D
:10A340002BD13B0000F0E7F90906090C4D114D4DEA
:10A350004D274D00FDF7D8F809E0FDF7E5F806E0D8
:10A360000968C90605D4304603E0FDF7EDF800287A
:10A370003DD0616840004A088018FAF7B9FE80B203
:10A380000146244A103991422BD8511C0140000744
:10A39000400F084329E01046EBE73B0000F0BBF913
:10A3A0000906090C2112212121232100FDF7ACF817
:10A3B0000AE0FDF7B9F807E00968C90606D4304697
:10A3C00004E00EE0FDF7C0F8002810D061684A08EC
:10A3D0001018FAF78DFE80B201460E4A10399142EC
:10A3E00003D9012503E01046F0E72168C86000208A
:10A3F0006066A0662846F8BD00480040F369FFEF9C
:10A4000000380140401002400044004000093D0077
:10A41000FFFC0F00EFFF0000F8B504464165403037
:10A4200000262746028380373E602220E0672546CB
:10A43000206F603500281CD01749C162216F174872
:10A440000863216F16484863206F8663236F606D31
:10A450009C4613462168024660462431FCF73CFACC
:10A46000002806D0102038602E752020A06701201B
:10A47000F8BD2E7520680168FF220132114301608A
:10A480002068816801221143816020688168402230
:10A49000114381600020F8BDF9A0000857A1000811
:10A4A000ADA00008FFB581B005460F4604466035F3
:10A4B0000A9E39E0701C37D0FCF7B6FB0499401AAD
:10A4C000B04222D8002E20D02068016849072BD541
:10A4D000C069C043000527D401202168C00208627A
:10A4E00020680168FF22A1329143016020688168E1
:10A4F0004908490081602020A067E067803420601F
:10A5000000202875032005B0F0BD20680168FF22F7
:10A51000A132914301602068816849084900816047
:10A520002020A067E067EBE72068C16938468843D0
:10A5300005D0002103988142BCD00020E3E701212F
:10A54000F8E7000010B504491020096808620248C5
:10A55000FDF7BAFC10BD00008C16002001490D204B
:10A56000887070475400002010B507480A22418ABD
:10A5700051438184FEF74AFAFEF762FBC822034981
:10A580000348FDF751FE10BD1C010020100D0020F6
:10A590008C160020F8B53E4C002321783D4A1D461C
:10A5A000082910D0072947D0062950D0052952D0B4
:10A5B000042953D0032954D0002956D0012958D05A
:10A5C00002295AD05BE0A17800264A1F04E0314FEF
:10A5D000BF5DFB189BB2761C9642F8DB6679277943
:10A5E0009A195118E3786278C9188918C91940185E
:10A5F000C0430006000E1AD1012E14D0022E16D12F
:10A6000025482449C018FAF7B9FD01F08BFF6420F2
:10A6100000F0A6FABFF34F8F21492048C860BFF36E
:10A620004F8F00BFFDE759081046FFF7A1F92570CD
:10A63000E570A570A571F8BDA1795054491CC8B248
:10A64000A071A178491F8842F5D1082001E060700F
:10A6500007202070F8BDE0700620FAE76071052041
:10A66000F7E7A070E5700420F3E7552807D1012033
:10A67000EFE7AA2803D10220EBE7032803D02570D7
:10A68000E570A570F8BD032020702071F8BD0000B2
:10A6900014010020A0140020D80D00200400FA05A9
:10A6A00000ED00E010B5024A024900F0E5F910BDE6
:10A6B00061B80008780100202021020C01D010218F
:10A6C0001046020A01D010460839020901D010468E
:10A6D000091F820801D01046891E420801D0881E39
:10A6E0007047081A7047F8B5040C8BB2264682B240
:10A6F0005E430D0C1046370C584336048019002178
:10A70000794116466E43370C360480197941264646
:10A710006E438919F8BD30B47446641E2578641CF4
:10A72000AB4200D21D46635D5B00E31830BC1847A6
:10A730004900CA020243100000D004204A0D01D093
:10A7400001221043044A490D914201D102210843DC
:10A75000012800D105207047FF0700008307FF2272
:10A76000DB0E9A408907090E9940002808DB830810
:10A7700009489B001B1818689043084318607047ED
:10A780000007000F0838830804489B001B18D8698D
:10A7900090430843D861704700E400E000ED00E01A
:10A7A000BFF34F8F04490348C860BFF34F8F00BF0A
:10A7B000FDE700000400FA0500ED00E0F8B50446EE
:10A7C0004F1EC8000838211815461E4608684968FB
:10A7D0003A4606239A4310D02A463346FAF792FEA9
:10A7E0003A46D200083AA3181A687F1E5B68FAF747
:10A7F000D7FD06223B469343EED1022F23D0042FF0
:10A8000011D0062F2FD12A463346FAF77BFEE36A92
:10A81000A26AFAF7C5FD2A463346FAF773FE636A61
:10A82000226AFAF7BDFD2A463346FAF76BFEE36962
:10A83000A269FAF7B5FD2A463346FAF763FE636963
:10A840002269FAF7ADFD2A463346FAF75BFEE36864
:10A85000A268FAF7A5FD2A463346FAF753FE636865
:10A860002268FAF79DFDF8BD002210B51346104688
:10A870000149FAF7AFFE10BD0000F03F10B5FAF73E
:10A880008FFD10BD002210B5134610461146FAF791
:10A89000A1FE10BD10B50721024A00200907FAF7F2
:10A8A00011FF10BD01030000034A10B5002011077D
:10A8B000FAF708FF10BD000001FDFFFF02E008C825
:10A8C000121F08C1002AFAD170477047002001E02A
:10A8D00001C1121F002AFBD1704700000149086026
:10A8E000704700007C01002008B500216846017017
:10A8F0006B46012202212C2000F052FF0221684603
:10A9000001706B4601222C2000F04AFF08BD0000B8
:10A9100038B504466D20694608706B460122074928
:10A920002E2000F03DFF0649002C01D0054A00E032
:10A93000054A2E2000F01AFF38BD0000060800006E
:10A9400006180000070600000716000038B5044688
:10A950006B4602220021362000F0EEFDB3212300D9
:10A96000FFF7D9FE0E0F08153A3A3A3A1C273A3A41
:10A970002F34483A00216846017040784108490068
:10A9800014E06946087880088000401C04E06946AD
:10A99000087880088000801C08701DE068460278F6
:10A9A0000A40483202704178802001436846417075
:10A9B00012E0684602780A40027040784106490E6B
:10A9C000F4E7694648780221084303E0694648787D
:10A9D000FD210840694648706B460122002136205F
:10A9E00000F0DEFE012200AB11463620013300F0FC
:10A9F000D7FE38BD69460878CF2108406946203027
:10AA0000CAE708B5032168464170012101706B4611
:10AA100002220021362000F0C3FE0122D2030621CB
:10AA20002D2000F0A3FE012000F09AF80120FFF78E
:10AA30008DFF08BD08B5020A69464A7008706B466A
:10AA4000022204212D2000F0ABFE0320694608708D
:10AA50006B46012206212D2000F0A2FE002069464F
:10AA600008706B46012206212D2000F099FE0A2174
:10AA70002D2000F047FD08BDF8B516460F460446E8
:10AA8000002503E03946B047641C6D1C207800287F
:10AA9000F8D12846F8BD0000F8B54A002B4B520DFE
:10AAA000D6182B4A0C460546142E2BDA002E12DA45
:10AAB000284BFAF775FC00221346FAF7E5FE40D260
:10AAC000002C03DA0124E40700253AE0204628435D
:10AAD00037D0214C14E0214F0B46F7403B402B432D
:10AAE00031D01C4BFAF75CFC00221346FAF7CCFE7F
:10AAF00027D2002C03DD01200005F0400419BC43DF
:10AB000000251EE0332E1EDC33460027143BFF4396
:10AB1000DF40384217D00F4BFAF7ECFC0022134607
:10AB2000FAF7B2FE0DD2002C0ADD142E0CD0342020
:10AB3000811B012088404019A84200D2641C0546B0
:10AB4000BD4321462846F8BD641CF9E701FCFFFF20
:10AB50009C7500883CE4377E0000F03FFFFF0F004B
:10AB60007D2110B5C900484300F001F810BD002157
:10AB700040E000BF00BF00BF00BF00BF00BF00BF7C
:10AB800000BF00BF00BF00BF00BF00BF00BF00BFCD
:10AB900000BF00BF00BF00BF00BF00BF00BF00BFBD
:10ABA00000BF00BF00BF00BF00BF00BF00BF00BFAD
:10ABB00000BF00BF00BF00BF00BF00BF00BF00BF9D
:10ABC00000BF00BF00BF00BF00BF00BF00BF00BF8D
:10ABD00000BF00BF00BF00BF00BF00BF00BF00BF7D
:10ABE00000BF00BF00BF00BF00BF00BF00BF00BF6D
:10ABF00000BF491C8142BCD37047FFB581B01E46DF
:10AC00000F46040026D00B9903980143A06A3943EC
:10AC1000826807209047002818DB0A99A06A314310
:10AC2000826806209047002810DB25462035A97948
:10AC3000032F01D908200143032E01D90420014329
:10AC4000A06A826809209047002806DA0120C043E4
:10AC500005B0F0BD0020C043FAE7384600F000F927
:10AC60002060304600F0FCF860600A986870039835
:10AC7000A870EF702E710B9868710020E8E7000053
:10AC8000F7B50446002090B000900190002C05D04C
:10AC90006A46062101F080FC062803DA0020C04342
:10ACA00013B0F0BD684640780102684600780004A1
:10ACB0000918684680780818FAF740FD0546684686
:10ACC0000391007901026846C078000409186846BB
:10ACD00040790818FAF732FD032206460F4692071C
:10ACE0005C4BFAF7D1FD07D200225B4B3046394668
:10ACF000FAF7FAFB06460F4603229207554B284601
:10AD00000399FAF7C1FD07D20022534B2846039955
:10AD1000FAF7EAFB054603912068FAF70FFD0246B1
:10AD20000B4630463946FAF755FC07460A2007918C
:10AD3000205EFAF7EFFC3A46079BFAF7E3FB06467C
:10AD400008200991205EFAF7D3FC0021C943FAF7E5
:10AD50001AFBFAF771FD3246099BFAF721FB0691BF
:10AD600008906068FAF7EAFC02460B462846039909
:10AD7000FAF730FC05461A200E46205EFAF7CAFCA8
:10AD80002A463346FAF7BEFB0C9009911620205E46
:10AD9000FAF7C0FC099B0C9AFAF702FB05910A909E
:10ADA0002A46334638460799FAF7ACFB059B0A9AC0
:10ADB000FAF7A8FB05910A901420205EFAF7AAFC86
:10ADC0003A46079BFAF79EFB07461C200791205E38
:10ADD000FAF7A0FC2A463346FAF794FB0E900B9143
:10ADE0001820205EFAF796FC0B9B0E9AFAF7D8FA19
:10ADF0002A463346FAF786FB0B910E902069FAF744
:10AE000089FC0B9B0E9AFAF7CBFA2A463346FAF7DF
:10AE100079FB05460E46E068FAF77CFC2A46334685
:10AE2000FAF7BEFA3A46079BFAF7BAFA059B0A9A6E
:10AE3000FAF7B6FA01229207084BFAF763FB0246CB
:10AE40000B46129C0898069903C411980CC0002068
:10AE500026E70000FFFF5F4100007041E17A843F78
:10AE600000B50121C9040300FFF755FC081A0508C5
:10AE70000B0E1114171A0320C00400BD0720C004D4
:10AE800000BD0F20C00400BD1F20400300BD3F20B7
:10AE9000400300BD7F20400300BDFF20400300BDF4
:10AEA000084600BDFEB5264F0D4604000FD0002D0C
:10AEB0000DD0264600202036B071F07129680D2093
:10AEC0008847002801DA7800FEBD102801D03846F6
:10AED000FEBDA562E968002901D0282088472046E8
:10AEE00000F030F80028F3DBA06AA52182680E206C
:10AEF0009047A06A962182680F209047A06A02219D
:10AF0000826862209047A06A002182680E209047E4
:10AF1000A06A002182680F2090477179302001914A
:10AF200000900623202201212046FFF766FE00281C
:10AF3000CEDB204600F0AEF80028C9DB0020FEBDC5
:10AF4000FFFFFFFF10B586B0044614216846FAF7EC
:10AF50002EF9002C7ED0A06A122143686A46102088
:10AF60009847122877D16846007801220101684687
:10AF7000407812030009081843492081884201DD06
:10AF8000801A20816846837840780007000D1818E1
:10AF90006081884201DD801A608168460079012263
:10AFA00001016846C0781205000309186846407917
:10AFB000000908183549E060884201DD801AE06028
:10AFC000684640790007030B6846807900021B1829
:10AFD0006846C07918182061884201DD801A206116
:10AFE0006846417A007A0002081802B22848012116
:10AFF0000904A282824201DD521AA2826A46D37AF1
:10B00000927A12029A1812B2E282824201DD521A38
:10B01000E2826A46537B127B12029A1812B2228392
:10B02000824201DD521A22836A46D37B927B12024E
:10B030009A1812B26283824201DD521A62836A4612
:10B04000537C127C12029A1812B2A283824204DD4F
:10B05000501A01E00BE008E0A083A06A01682820F4
:10B060008847002806DA0120C04306B010BD002042
:10B07000C043FAE7C011C0072034002800D0802068
:10B0800060710020F1E70000FF070000FFFF0700EC
:10B09000FF7F000010B5040009D0A06A0721826874
:10B0A00008209047002805DA0120C04310BD002089
:10B0B000C04310BD072020342070002010BD0000C8
:10B0C000FEB504460020019000906079734940006D
:10B0D0000E5A61782578491E7148CFB20163042D5C
:10B0E00077D0072D75D000210291217801736C492A
:10B0F000E379012292058969002B6CD0914381612B
:10B100006748217A4173217A82698907890B0A434A
:10B1100082610021042000F034FB324661492E2078
:10B1200000F024FB3846FFF7F3FB5F4E0522705D0D
:10B13000810040185D49431807212B2000F030FBA7
:10B140005B49029801220B180B21282000F028FBF4
:10B15000705D584980000A580C21282000F011FB2E
:10B16000E079554980004018A1794900425A0221EE
:10B17000272000F0FBFA51487E00825B0421272043
:10B1800000F0F4FAE079002829D0A07804282CD027
:10B1900028206946087220220621272000F0E6FABE
:10B1A00002AB01222621272000F0FAFA4449380197
:10B1B0004018E178890042580821272000F0E1FA80
:10B1C000A17A601C627A0902114313D016E000E0F4
:10B1D00001E0012188E71143F608816190E76422CC
:10B1E0000621272000F0C2FAE0E710206946087225
:10B1F0000246D1E733490172090A4172417A007A65
:10B200000A0202432021272000F0B0FA2E4F0C2121
:10B2100023203A6800F0B5FAF0198288042123202F
:10B2200000F0A4FAA07900280BD0E0792749012288
:10B2300043180021212000F0B3FA032001900120DF
:10B2400000902A07120F1001024360780021800746
:10B25000000B02430198000502430098400402439A
:10B260002079C006400902436079C00602431F20CE
:10B2700000F087FAA07861780123084302040848A7
:10B28000DB030261E179490319430A4302610021AA
:10B29000082000F076FA0020FEBD0000CCC60008B1
:10B2A000AC0100200428000074C60008240000201F
:10B2B000420000207CC600089CC60008A8C6000802
:10B2C000ACC600084110000094C6000844000020ED
:10B2D00038B50C4607498A8B002102432C2000F028
:10B2E00045FA684604706B46012206212C2000F0C6
:10B2F00057FA38BDAC01002010B5FFF7F5FA10BDC4
:10B3000010B504460421362000F0FCF80121C902E2
:10B31000002C01D0084300E0884302460421362077
:10B3200000F02FFA10BD000038B5402069460870C3
:10B3300000210E2000F0E6F80446002211460E20FF
:10B3400000F01FFA6B46012200210D2000F028FAC0
:10B35000074A00210F2000F014FA00F0EDF9224610
:10B3600000210E2000F00DFA02480021017338BDC3
:10B37000F8FF2724CC010020FEB5054604206946CD
:10B380000870514C002060752146203120634871BF
:10B390000873A0836063A06300F0C8F84B4E206080
:10B3A00002E000F0C3F82060B042FAD10020FFF7BD
:10B3B000CDFA00F0BBF8464E20603078242801D941
:10B3C000243806E00621F9F793FE0622101A400100
:10B3D0000843020601040A4301020A430243B26021
:10B3E000706000211E2000F0CCF900F09FF8206072
:10B3F0006B4601220021242000F0D2F91E20FFF725
:10B4000019FB86B2300AA0730420FFF713FB07462E
:10B4100000F08CF820603806000E0DD0022069463E
:10B42000087101AB012212212D2000F0B9F9A08B87
:10B43000012109030843A08300F078F8206006206A
:10B44000FFF7F8FA60600720FFF7F4FAA060F00653
:10B45000C00E207501D110202075C0B200F0DCF9BB
:10B46000E80707D0FFF7CDFAA08B0121C9020843F6
:10B47000A0830AE00521362000F02EF81549084087
:10B4800002460521362000F071F90120FFF75EFA2F
:10B490000021042000F036F8A0610021262000F0F1
:10B4A00031F815218903084302460021262000F0C7
:10B4B00068F900222621362000F058F900F036F80D
:10B4C00020600020FEBD0000AC0100203001CADE7B
:10B4D00018000020FFFD000038B5094C89B280B289
:10B4E0006B46022200F028F8002806D16846407812
:10B4F000010268460078081884B2204638BD000072
:10B50000FFFF000038B50024E44389B280B26B46E7
:10B51000042200F011F8002806D103216846435C9C
:10B520002202D418491EFAD5204638BD10B5002194
:10B530000846FFF7E7FF10BD38B5002909D04024C1
:10B5400020436C462070C8B27F2906D86070022064
:10B550000AE069460870012006E0802420436C461A
:10B560006070C809A0700320694600F0B5FF38BDBF
:10B5700010B5144603460A4621461120FFF7DCFFAA
:10B5800010BD10B50346052200211520FFF7D4FF9A
:10B5900010BD10B50346052200211720FFF7CCFF90
:10B5A00010BD38B5054600206946087000F0C4F8A3
:10B5B000FF2401342246002D01D003221202002173
:10B5C0000D2000F0D3F8002D13D06B46012203218B
:10B5D0000F20FFF7B1FF68460078000709D5FFF795
:10B5E000A3FE224600210D2000F0C0F80020C04339
:10B5F00038BD002038BD10B5024601210A2000F0F8
:10B60000C0F810BD10B5044600211A20FFF77AFFDC
:10B61000000D22030005120B024300211A2000F046
:10B62000B0F810BD10B5024602492E2000F09EF879
:10B6300010BD000004180000F8B505466B46012255
:10B6400003210420FFF778FF0126114C3607002D57
:10B650000DD02A4600210C2000F088F869460878B1
:10B660001021084369460870A069304307E0694625
:10B670000878EF21084069460870A069B0430B467E
:10B68000A06101220321042000F08AF8F8BD000027
:10B69000AC01002010B502460021182000F066F829
:10B6A00010BD0000F8B50746002568460570B807CC
:10B6B000204C2E4600280ADA8020694608706B4626
:10B6C000012200210D2000F06BF801202073F80703
:10B6D0006946087821D006210843694608706B4600
:10B6E000012200210D2000F05BF803210F20FFF75D
:10B6F000F3FE8121C900084219D040206946087034
:10B700006B46012200210D2000F04AF80020FFF7CF
:10B71000F7FD00252673ED4309E002210843694641
:10B7200008706B46012200210D2000F039F82846F0
:10B73000F8BD0000CC0100201CB56B46012203219E
:10B740000F20FFF7F9FE684600784022C10910403B
:10B75000C9014000814208D00120694608710246B3
:10B7600001AB03210D2000F01BF81CBD08B56B4692
:10B770001A70120A5A7089B280B2022200F010F8D0
:10B7800008BD38B500236C46E254120A5B1C042B3A
:10B79000FADB89B280B22346042200F001F838BDFA
:10B7A00038B58024002909D0C02528436D4628706B
:10B7B000C8B27F2907D86870022009E02043694693
:10B7C0000870012004E020436870C809A8700320B5
:10B7D000694600F02BFF38BD10B51446012312183E
:10B7E0009B029A4202D90020C04310BD0B46821E24
:10B7F00021460920FFF7D4FF002010BD10B5054AEF
:10B800008905126901430A4300210820FFF7B9FFA7
:10B81000002010BDAC01002038B504466B46012263
:10B820000E212B20FFF788FE68460078E1064009CC
:10B830004001C90E0143684601706B4601220E218A
:10B840002B20FFF7ADFF38BD10B5002142541C0678
:10B85000120A22431B0A491C0429F7DB10BD000011
:10B8600013B501231A4669460248FCF70FFD0098FC
:10B870001CBD00008C1600207CB5002425466846BF
:10B88000FFF77FFE04206946220E2D021543220297
:10B890000C5C1443401EF7D5204629467CBD7CB580
:10B8A000002425466846FFF774FE04206946220EF0
:10B8B0002D02154322020C5C1443401EF7D520468E
:10B8C00029467CBDFBF7BEF9FEF7EAF8FDF7B2F8B2
:10B8D00040494148002522C005608561C5613F4956
:10B8E0000562C1600838FBF749FBFDF78FF8FDF7EB
:10B8F000A7F9FDF743F9FDF755F8052601223607AC
:10B90000D1033046FBF789F9FDF730FEFCF73EFF27
:10B91000FAF720FAFAF7EEF9FCF73AFD0721B0152D
:10B92000FFF7D6FCFFF7E8FC2D4C0A21608A0122C4
:10B930004843A08411033046FBF76FF92648C8221C
:10B940002849C830FCF770FC274F284E6079002842
:10B950003DD0A07800283AD0FEF7A2F86571207893
:10B960000F280AD9012211033046FBF756F9FEF7DA
:10B97000E5F900220121090309E0012251033046C3
:10B98000FBF74BF9FEF7DAF90022012149033046B3
:10B99000FBF743F9FCF724FEA08C002801D0401EE1
:10B9A000A0841348A18C00780843CFD138780028B0
:10B9B00001D00328CAD10121C9023046FBF720F982
:10B9C0000028C3D101210846FBF7ECFBBEE7FCF7DA
:10B9D00007FEBBE7007C0040C4150020FFFF00000D
:10B9E0001C010020100D00208100002000040050E8
:10B9F0005A00002010B586B01748FBF742FA142110
:10BA00006846F9F7D4FB1548009003200190002008
:10BA10000290052069460007FBF736F86946104892
:10BA2000FBF732F869460F48FBF72EF8012108466C
:10BA3000FBF7B8FBFF2401342046FBF78BFB0A49D8
:10BA400008680422104308602046FBF793FBFBF7CD
:10BA500099FB06B010BD0000C4150020FFFF0000D8
:10BA600000040050000800500070004010B5012292
:10BA7000920217491748FAF7F9F91548164902884A
:10BA80008A4224D00180FF2101318180FF21F531DC
:10BA9000C1800A21018100211E224181D24382817D
:10BAA0000122C28181831E23C38602230387782358
:10BAB00043878287C2870246403211845184918431
:10BAC000C183918014238382118200F02BFD10BD6D
:10BAD000D80D002000FC0008AA550000F0B51FB4E6
:10BAE00096B084460C460246199D1898039049006A
:10BAF00068006300490840080193002A01D001262C
:10BB000000E000269E19FE4BF6185B109E422BD3D8
:10BB10006E00039F0296002F00D00127F719F84E00
:10BB2000F84BBE199E421FD3039E0346F64F334384
:10BB300009D03B469C4201D1002A04D0019B002A37
:10BB400005D0012604E0002039461BB0F0BD0026D8
:10BB50009E19EE4B9E4207D8039F029E002F00D0F5
:10BB60000127F6199E4207D92B4660462146189AAE
:10BB7000FEF784FE1BB0F0BD0023002C29DAE44E52
:10BB8000B04226DAE34EB04201DB022321E0DE4E72
:10BB9000B0421EDBE04E070DBE19142E09DD34271E
:10BBA000BF1B039EFE400196BE40039FBE420BD0CA
:10BBB0000FE0039F002F0CD11427BF1B0646FE4049
:10BBC0000196BE40864204D1019BDE07F60F022398
:10BBD0009B1B0E46164318D1002D16DA002C03D0FD
:10BBE000022B01D0012B06D00220FEF777FEFEF7D4
:10BBF0003BFE1BB0F0BD0220FEF770FEFEF734FEE8
:10BC00000122D20751401BB0F0BD039E002E61D12E
:10BC1000BF4EB04220D1C148844201D1002A08D091
:10BC2000B948814209DB002D10DB189829461BB06A
:10BC3000F0BD0020B4491BB0F0BD002D06DA012292
:10BC40002946D207189851401BB0F0BDB449794439
:10BC5000086849681BB0F0BDAB4FB84225D1002D34
:10BC60001FDA002904D0B14212D1002A09D018E00D
:10BC7000002A72D1A649E20F0020D20711431BB05F
:10BC8000F0BD0020E20F0146D20711431BB0F0BD0A
:10BC9000B14206DA234600203946F9F79BFC1BB077
:10BCA000F0BD104621461BB0F0BDB14212DA0126AC
:10BCB000B607B54203D1234610461946FEE3994E16
:10BCC000B54207D1261E05DB1046314600F040FC88
:10BCD0001BB0F0BD67007F081646002A40D100293E
:10BCE0000AD08B4A914229D1002C0EDD002D1CDB9D
:10BCF000002011461BB0F0BD022B16D0002C14D032
:10BD0000012B12D1002C14DB0FE0002C28DA002DBF
:10BD100009DB012B03D000207D491BB0F0BD0020C2
:10BD200081491BB0F0BD012B03D0002001461BB0A0
:10BD3000F0BD00200121C9071BB0F0BD724A91423D
:10BD40000ED1002C01DA002B17D0022B06D00020D8
:10BD5000C043F9F7DFFC1BB0F0BD90E20120F8E72B
:10BD6000E217521C94461A4307D000220892664CF0
:10BD700062465B1E1A4307D009E00120FEF7AEFDC4
:10BD8000FEF780FD1BB0F0BD0022644C0892674AAC
:10BD900090427DDD664B674A98421FDD914202DC8E
:10BDA000002D05DB4DE05848814217DB002D48DDB2
:10BDB0000220FEF793FDFEF76DFD05460E460022BC
:10BDC000534B21460898F9F79DFB08467100490836
:10BDD000C00FC007014328461BB0F0BD914215DAE1
:10BDE000002D2EDA0220FEF779FDFEF753FD054601
:10BDF0000E460022464B21460898F9F783FB720055
:10BE00005208C80FC0070243114617E03E4B994243
:10BE100023DD002D15DD0220FEF760FDFEF73AFD63
:10BE200005460E4600223A4B21460898F9F76AFB70
:10BE3000084671004908C00FC007014328461BB0DF
:10BE4000F0BD0220FEF74AFDFEF72EFD490049082D
:10BE5000E20FD20711431BB0F0BD00223046394635
:10BE6000F9F742FB012205460E46D243F9F72AFCB8
:10BE7000314A324BF9F73EFB2A463346F9F742FB8B
:10BE80000022284BF9F736FB07462A46334600E0E6
:10BE900064E0039110461946F9F734FB3A46039BD8
:10BEA000F9F730FB0746032209915207244B284635
:10BEB0003146F9F727FB07910C90224A204B384670
:10BEC0000999F9F71FFB074601911F4A1F4B2846A6
:10BED0003146F9F717FB3A46019BF9F705FB074690
:10BEE0000B460246099107990C98F9F759FA002573
:10BEF0000E462846079B0C9AF9F7F6FA3A4627E0D1
:10BF0000FFFF1F00FFFF0F000000F03F0000E0FFF9
:10BF10000000F07F0000404301FCFFFF0000F0BF85
:10BF2000560B00000000E03F0000F0FF0000E04181
:10BF30000000F043FFFFEF3F555555555555D53F90
:10BF40004715F73FFE822B6544DF5DF80BAE543E8C
:10BF5000099BF9F7CFFA02460B4652E10125002072
:10BF60002D05A94207DA352230463946F9F7AAFBF2
:10BF700006463420C0430A151218FE4810180390D4
:10BF80000803FD49000B01430F46FC49884201DCD0
:10BF9000002003E0FA49884202DA0120119005E00E
:10BFA000002011900398401C7F1B03901198059767
:10BFB000C200F4480F9278448018436802683946FA
:10BFC00030460D930292F9F78FFA07910C903046A4
:10BFD0000D9B029A0599F9F7E3F902460B460020FA
:10BFE000E549F9F7F7FA09910490079B0C9AF9F7DC
:10BFF00089FA129000201090E3480D4678440068BA
:10C000000E90012178104907084311990D9B89046E
:10C0100040180121C90447183946029A0E98F9F7C9
:10C0200063FA3246059BF9F765FA02460B46294644
:10C030001098F9F767FA064602913B4629460E9A90
:10C040001098F9F75FFA079B0C9AF9F753FA324602
:10C05000029BF9F749FA099B049AF9F753FA0591FB
:10C06000129A0A902B4610461946F9F74BFA0646E3
:10C070000246C6480F460B4606217844FEF79EFB53
:10C0800032463B460091049010461946F9F73AFAB9
:10C09000009B049AF9F736FA06460F462B461946D6
:10C0A000129A1098F9F77CF9059B0A9AF9F72AFA7F
:10C0B00032463B46F9F774F9109A079104902B46E3
:10C0C00010461946F9F71EFAB14E0022334609917F
:10C0D0000290F9F765F9079B049AF9F761F90020D6
:10C0E0000746024633460091F9F7FEF9099B029A8A
:10C0F000F9F7FAF9079B049AF9F7FCF906460D914E
:10C100003A462946009B1098F9F7FCF907910C90E4
:10C110002B463046129A0D99F9F7F4F905460E466A
:10C120003A46009B05990A98F9F7ECF933462A46F6
:10C13000F9F736F902460B460746099107990C981C
:10C14000F9F72EF900250E462846079B0C9AF9F7B9
:10C15000CBF93A46099BF9F7CDF907460722099131
:10C1600052078C4B31462846F9F7CCF907910090DD
:10C17000894A884B38460999F9F7C4F9074601916D
:10C18000864A874B31462846F9F7BCF93A46019B67
:10C19000F9F706F9834B7B440F9A9B181A685B6882
:10C1A000F9F7FEF8029009910398F9F7B3FA0591AF
:10C1B0000490099B029A07990098F9F7F1F87A4BD5
:10C1C0007B440F9A9B181A685B6817460393F9F72C
:10C1D000E7F8059B049AF9F7E3F80E462846059B15
:10C1E000049AF9F781F93A46039BF9F77DF9079B21
:10C1F000009AF9F779F9099B029AF9F77BF9024657
:10C200000B46199900200C900F461898F9F77AF907
:10C21000029104903B460C9A19991898F9F764F921
:10C220002A463346F9F76EF9029B049AF9F7B8F8F3
:10C2300009910E902A46334639460C98F9F762F96F
:10C2400006460F46099B0E9AF9F7AAF8574A0D467B
:10C25000914220DB5242AA18024310D132463B469B
:10C26000F9F742F904900391514A524B09990E98FB
:10C27000F9F796F8039B049AF9F706FB1ED2022001
:10C28000FEF72CFBFEF706FB49004908E20FD20738
:10C2900011431BB0F0BD6A00474B52089A420DD3C0
:10C2A000464AAA18024300D0CBE532463B46F9F78E
:10C2B0001BF9099B0E9AF9F7E7FAF5D968000023F4
:10C2C00040082C490393020D3D4B5218984223DD40
:10C2D00001200005521CD04042195000400D40186A
:10C2E00038497944096813468C463749C1408B4325
:10C2F00012030121120B090551181422101AC14012
:10C300000391002D01DA48420390624630463946D7
:10C31000F9F7EAF806460F4632463B4609990E9869
:10C32000F9F73EF800252A46284B28460591F9F7EB
:10C33000E9F807910C90264A264B28460599F9F70B
:10C34000E1F80091029032463B4628460599F9F7FC
:10C35000CBF8099B0E9AF9F7CDF81F4A1F4BF9F756
:10C36000D1F8009B029AF9F71BF807460B460246E4
:10C37000099135E001FCFFFF0000F03F8E980300BB
:10C380007AB60B0066070000A8070000D20600007E
:10C390000000084009C7EE3FFD033ADCF5015B14DD
:10C3A000E02F3EBEA60500006C0500000000904096
:10C3B000FE822B654715973C00CC904000346F3FC0
:10C3C0000000E03FC2040000FFFF0F00432EE63FE5
:10C3D000396CA80C615C20BEEF39FAFE422EE63FB4
:10C3E00007990C98F8F7DCFF05460E46079B0C9A58
:10C3F000F9F77AF83A46099BF9F77CF809912A4649
:10C4000033460E9010461946F9F77CF80746024667
:10C410002F480B46059105217844FEF7CFF93A469F
:10C42000059BF9F76FF82A463346F9F763F8074694
:10C43000019128463146099B0E9AF9F763F8099B4A
:10C440000E9AF8F7ADFF012304910C9000229B0790
:10C4500038460199F9F748F805910E903A46284672
:10C460003146019BF9F74EF8059B0E9AF9F7B2F8A1
:10C47000049B0C9AF9F738F82A463346F9F734F852
:10C480000022144BF9F736F8064603980D460005CE
:10C4900041190915002912DC30462946039AF9F79B
:10C4A00011F9FEF745F9042801D1FEF7FDF93046F0
:10C4B0002946039AF9F706F9064601E004E029182F
:10C4C0000B46324621460898F9F71CF81BB0F0BD20
:10C4D000640300000000F03FF0B58C4600251026F4
:10C4E000052109078E620E4C08E067467F5DE76014
:10C4F000A768FF07FCD0E7681F706D1C8542F4DB5E
:10C500000020074606E0E760A568ED07FCD0E56877
:10C510001D54401C9042F6D38E610020F0BD0000F7
:10C520000030014070B572B60124074DA4022146C7
:10C530002846F9F781FC002804D022460349284602
:10C54000F9F71EFD62B670BD00FC0008D80D002092
:10C55000F8B506460C46F9F7A5FA051E0F4600D0B9
:10C560000120014349000B484908411AC90F0DD069
:10C57000002E01D0012100E000210C436100490898
:10C58000401AC00F02D10120FEF7A8F9284639460B
:10C59000F8BD00000000F07FF8B515460E460746CE
:10C5A000002407E03819C0B200F008F8641C2870B5
:10C5B000E4B26D1CB442F5D33046F8BD10B5044664
:10C5C000FBF7AAFFEE20FBF77AFFFBF7DEFF204622
:10C5D000FBF775FFFBF7D9FFFBF79EFFEF20FBF79B
:10C5E0006EFFFBF7D2FF0020FBF73CFF0446FBF792
:10C5F000AEFF204610BD704770B50D460446FBF7F0
:10C600008BFFEE20FBF75BFFFBF7BFFF2046FBF73E
:10C6100056FFFBF7BAFF2846FBF751FFFBF7B5FFC4
:10C62000FBF795FF0A20FEF7A2FA70BDF0B50025D2
:10C63000102605279C463F070B46BE620C4C06E0C1
:10C64000595DE160A168C907FCD0E1686D1C8542B5
:10C65000F6DB002007E06146095CE160A168C907DC
:10C66000FCD0E168401C9042F5D3BE610020F0BDD3
:10C67000003001400000010203040005405C00009E
:10C68000A05C0400C06C0800805C0400E03F1E0059
:10C69000E07D1E0007A9022570889B880A0016000D
:10C6A000010006000100020087008D002D001A31F4
:10C6B00052001A339A001A351D011A376B003B31AC
:10C6C000BE003B335E013B3596023B370000995973
:10C6D0009959EB518F421E45142E0080EB51F528DD
:10C6E0003333E13A703DE13AC235852BC2353333FD
:10C6F000C235C235AE47E13A5138A3305138000057
:10C7000000000000000001020304060708090304FA
:10C7100006080C101820300000000001020304007D
:10C72000000000000000F03F000000000000F83FA3
:10C7300000000000000000000000004003B8E23FDD
:10C74000000000000000000006D0CF43EBFD4C3E8F
:10C75000033333333333E33FFFAB6FDBB66DDB3F84
:10C760004D268F515555D53F01411DA96074D13FCC
:10C7700065DBC9934A86CD3FEF4E454A287ECA3FC6
:10C780003E5555555555C53F93BDBE166CC166BF48
:10C790002CDE25AF6A56113FF16BD2C541BDBBBE41
:10C7A000D0A4BE726937663E0000000000000000A1
:10C7B000D0C7000800000020800100006C5B00086A
:10C7C00030C8000880010020381A0000CCA80008FA
:10C7D0000124130704380D091E0805400826091016
:10C7E0004008560A131D043B08BE0516D8BC40106D
:10C7F0000852010336C84203585C121B0202BD14E2
:10C800000901022281F01F66810498899686967933
:10C81000821598039814988796749778824397881E
:10C82000967197778229D1024A04C94F922000005D
:04000005080050C1DE
:00000001FF
